:1000000000400020CD6600000D6700000F67000073
:1000100000000000000000000000000000000000E0
:100020000000000000000000000000001167000058
:1000300000000000000000001367000015670000CA
:1000400017670000253B0000F16A000017670000F9
:100050001767000000000000176700001767000026
:1000600017670000C96D00001767000017670000E0
:100070001767000017670000176700001767000088
:10008000176700002D6F000017670000176700005A
:100090001767000017670000176700001767000068
:1000A0001767000017670000000000000000000054
:1000B0000000000000000000000000000000000040
:1000C000054B0648033310B51B1A062B03D9044B06
:1000D000002B00D0984710BDAC020020AC020020DD
:1000E000000000000648074910B5091A8910CB0F17
:1000F0005918491003D0044B002B00D0984710BD6D
:10010000AC020020AC0200200000000010B5074C3B
:100110002378002B09D1FFF7D3FF054B002B02D02A
:10012000044800E000BF0123237010BDAC02002092
:1001300000000000F8B20000094B10B5002B03D0FE
:100140000849094800E000BF08480368002B02D1B5
:10015000FFF7C8FF10BD064B002BF9D09847F7E713
:1001600000000000B0020020F8B20000A802002049
:1001700000000000164B002B00D1144B9D4640227E
:1001800092029A1A924600218B460F461348144A4F
:10019000121A08F0AAFD0F4B002B00D098470E4B07
:1001A000002B00D098470020002104000D000D48CE
:1001B000002802D00C4800E000BF08F053FD2000EA
:1001C000290006F0ADFC08F027FDC046000008003D
:1001D000004000200000000000000000AC020020F1
:1001E00090260020000000000000000001230340D2
:1001F0000200181E04D1042A03D91068000900E087
:100200000020704710B50400FFF7F0FF0300002046
:1002100083420BD0013B9B00181DE2181279002A83
:1002200003D001338342F8D100E0180010BD012251
:10023000096810B5114201D0002903DA102000F03E
:1002400083F903E04910062002F0ACF810BD0968FC
:1002500010B5CB0701D5002903DA102000F074F99E
:1002600006E04910033189100022052002F09AF8B7
:1002700010BD70B50D68AB0728D1042D26D90F230A
:100280002A684E681340062B09D12800FFF7AEFFFD
:10029000012383421DDC9A00AE500133F9E7052BA0
:1002A00014D1F30703D4132000F04EF912E07610B6
:1002B000FF2EF8D82800FFF799FF2C1D230080009F
:1002C0002018984205D91E700133FAE70B2000F080
:1002D0003BF9002070BD70B50C681120E3072DD5E7
:1002E0004D68AB0729D1042D27D90F262B68641040
:1002F0001E40062E0BD1002C04DD2800FFF776FFF0
:10030000844201DD122019E0A400605918E0331F77
:10031000012B12D82800FFF769FF8000042E02D1BC
:100320002800FFF76FFF002CECDDA042EADB012381
:100330002C19E0784000184302E00B2000F004F98B
:1003400070BDF8B501230C6811201C422FD0032585
:100350004E6835402AD1042E28D90F233268641004
:100360008F681340062B0BD1002C04DD3000FFF703
:100370003DFF844201DD122019E0A400A75113E0E3
:10038000052B13D1002CF6DD3000FFF72FFF800086
:100390008442F0DC01231F4201D1132007E07F10CB
:1003A000FF2FFAD83419E770280002E00B2000F084
:1003B000CBF8F8BD086810B5830717D1042815D904
:1003C0000F2302681340062B02D1FFF70FFF0BE04B
:1003D000052B05D1FFF70AFFC0000123184308E0F1
:1003E000042B03D1FFF70EFF4000F6E70B2000F0CF
:1003F000ABF810BD012303400200181E01D05010BD
:1004000002E00D22014B1A707047C046C80200205E
:10041000012303400200181E04D1042A03D91068E6
:10042000000900E00020704770B50D000400FFF7E0
:10043000EFFF86002800FFF7EBFF830000209E42BD
:100440000ED1231D9E1904351A009E4207D9297822
:100450001278013301358A42F6D0002000E00120F5
:1004600070BD0000F0B585B00393019002912D4E50
:100470002D4B002A02D002223270013A00251A6068
:100480001B68F554019B9D424ADA029AAB00D05892
:10049000254B1C68C8239B0037191C1B01231842DD
:1004A00002D04310214A1FE0214A002802D004282C
:1004B00005D1204A2100380008F0DEFF18E00428AA
:1004C00010D90F2302681340042B04D101F0A6FFBA
:1004D000194A030008E0062B05D1FFF799FF174AD8
:1004E000030001E00123164A2100380008F0C4FF90
:1004F000300009F027F8039B0B4A002B01D1106054
:100500000CE0019B013B9D42F9DA0E4B9842F6DC70
:10051000431C1360202232540022F2540135B1E70B
:1005200005B0F0BDD4020020D002002069A2000076
:100530003CA2000042A200005AAC000047A200000A
:1005400058A200001F030000014B187000207047E4
:10055000C802002070B501F07FFD094C0100251D87
:100560001F22280008F0F5FF280008F0EBFF042305
:1005700004308008000118432060200070BDC04690
:10058000F4050020C368F0B59D00836889B05D194B
:10059000030018330693036903909E00069B9F197E
:1005A00043699E000193069B9E19CB4B1B78002B41
:1005B0000FD17F222B68C9491C1213409B005B5846
:1005C00001960435029235E0C34B1B78002B29D0ED
:1005D000019E039BC04C9B6821780193EA1A039B00
:1005E00092109B7812021A43039B587803F02AFF5B
:1005F0000023039A2370137001960497039B069AB5
:100600009B680293ED1A039BAD10DD60049B9F1A5B
:10061000039BBF101F61019B9B1A039A9B105361A0
:1006200009B0F0BD2B68029A1C121340AB4A9B0024
:100630009B5804359F46039B587803F0FBFE00232C
:10064000039A1370D9E7069B3A1DD11AA24BDB29F6
:1006500003DD1A22019E1A70BBE71B783C60002B59
:1006600002D0019E1700B4E72B6802991C120B40C0
:100670009A499B005B5817000435DBE7069B3A1D3F
:10068000D11A954BDB2903DD1A22019E1A70A0E7CF
:1006900028681B78291D3860002B03D0019E1700A5
:1006A0000D0096E76B6802991C120B408B499B006A
:1006B0005B5817000835BDE7069B3A1DD11A864BDB
:1006C000DB2903DD1A22019E1A7082E7A4001B7841
:1006D0002C193C60002B02D0019E170079E72B6893
:1006E00002991C120B407D499B005B581700043592
:1006F000A0E7069B3A1DD11A774BDB2903DD1A22AE
:10070000019E1A7065E77648A40021581B7839606D
:10071000002B02D0019E17005BE72B6802991C1288
:100720000B406E499B005B581700043582E7043F7D
:100730006B4B3A68A400E250674B1B78002B01D04A
:10074000019E46E72B68029A1C121340634A9B00E5
:100750009B5804356EE7624BA600F058FFF74AFE3F
:10076000043F04003868FFF745FE241801205C4B65
:1007700064000443F450584B1B78002B01D0019EB9
:1007800027E72B68029A1C121340544A9B009B587F
:1007900004354FE7069B3A1DD11A4F4BDB2903DD89
:1007A0001A22019E1A7014E70198069C0121A042AA
:1007B00002D901000C3909681B783960002B02D07E
:1007C000019E170005E72B6802991C120B40434954
:1007D0009B005B58170004352CE7069B3A1DD11A85
:1007E0003D4BDB2903DD1A22019E1A70F1E60199C7
:1007F000069881420AD90B000C3B1B6839495B10F3
:100800006418E41A019BA400E35802E0182119704F
:1008100000233B60304B1B78002B02D0019E170059
:10082000D7E62B6802991C120B402C499B005B58A1
:1008300017000435FEE6019B069A93420CD90C3B47
:100840001968284B3E1FE3184910591A3268019B5A
:100850008900CA50370002E018221F4B1A701E4B45
:100860001B78002B01D0019EB3E62B68029A1C1264
:1008700013401A4A9B009B580435DBE6019B069AFD
:10088000934220D9174B3E1FE318019C04930C3C64
:100890002368049A5B10D31A019A9B009858FFF7BB
:1008A000A9FD07903068FFF7A5FD2468049B64103C
:1008B0001C1B079BA4001F1801207F00019B0743FE
:1008C000E750370002E01822034B1A70024B1B78E6
:1008D000002B09D0019E7CE6C80200207CA200000B
:1008E000D4230020FDFFFF3F2B68029A1C12134007
:1008F000CD4A9B009B5804359CE6069B3A1DD11AB5
:10090000CA4BDB2903DD1A22019E1A7061E60199A8
:10091000A40061581B783960002B02D0019E17009B
:1009200057E62B6802991C120B40BF499B005B588D
:10093000170004357EE6043F019B3A68A400E250AC
:10094000BA4B1B78002B01D0019E42E62B68029A1D
:100950001C121340B44A9B009B5804356AE6019B65
:10096000A4001C192368043F38685E10FFF742FD9D
:1009700036180120AD4B76001B7806432660002B0D
:1009800001D0019E25E62B68029A1C121340A64A4C
:100990009B009B5804354DE6069BA4003F1BA34CCF
:1009A000BB420DD82378002B01D0019E11E62B68A5
:1009B000029A1C1213409C4A9B009B58043539E64E
:1009C0009B4801F09FFC2378002B01D0019E00E69C
:1009D0002B68029A1C121340934A9B009B580435C3
:1009E00028E6A300ED18002C00DA06E68F4B1B78F2
:1009F000002B01D0019EECE52B68029A1C121340DB
:100A0000894A9B009B58043514E63B1F04931B68DE
:100A10000793042B04D1A300ED18002C00DAEDE5B8
:100A2000824B1B78002B02D0019E049FD1E52B68DE
:100A3000029A1C1213407C4A9B009B58049F043569
:100A4000F8E53B1F04931B68042B06D0A200AD18E9
:100A5000002C02DA002B00D1D0E5744B1B78002B60
:100A600002D0019E049FB4E52B68029A1C12134029
:100A70006D4A9B009B58049F0435DBE53A1F1368C1
:100A80005B10013B002B07DD01215B00A4000B4341
:100A900004972D191360B1E5644B17001B78002BE8
:100AA00001D0019E95E52B68029A1C1213405E4A04
:100AB0009B009B580435BDE53A00069B0C32D31AC7
:100AC000DB2B04DD1A22594B019E1A7081E5FF23AE
:100AD00061005B000B4001210B433B60039B0698C8
:100AE0009B6824120493ED1A039BAD109B782D0292
:100AF0001D43019B8D401B1A9B108B400B43BB6019
:100B0000039B0D437D609C70E4B24A4BE400039963
:100B1000E35816008B6045490978002903D0083353
:100B20001D00170055E51D0002999B680C351C122D
:100B30000B403D499B005B58019217007AE53B1F33
:100B40001C68069A019B93422AD104970A20E30766
:100B500016D4A3070DD1042C0BD90F232268134000
:100B6000042B06D1200001F059FC08F0EBFC063004
:100B700006E00720042C03D0002C01D08020800048
:100B8000643003F05BF9002801D1043D36E5039B96
:100B90002100587803F068FC0023039A13702DE5B8
:100BA000019B019A0C3B1B6803995B109B005B4205
:100BB0001E00D3180C3B1C601300083B1B68083E4A
:100BC00097195A108A70D2B21A49D2005B00555850
:100BD0009B0A039A9B009560ED18019B043B1E68DD
:100BE000069B7610B6009E19104B1B78002B00D088
:100BF000EFE42B68029A1C1213400B4A9B009B588F
:100C00000196043516E53B1F1868FFF7F3FBA400B7
:100C100006003F1B1E2831DC002816DC034B1B7826
:100C2000002B09D0019ED4E47CA20000C802002061
:100C30006CA20000DC1B00202B68029A1C121340DF
:100C4000C54A9B009B580435F4E401F0EBF9033EE0
:100C5000361801F0E7F9C14B801B9842F9D8C04B18
:100C60001B78002B01D0019EB3E42B68029A1C1262
:100C70001340B94A9B009B580435DBE40123039AD7
:100C8000137001F0CFF9039B0A3886195E60B4E453
:100C90003B1F1868FFF7AEFBA40004903F1B002821
:100CA0000EDCAF4B1B78002B01D0019E91E42B682A
:100CB000029A1C121340A84A9B009B580435B9E4C1
:100CC000A84B049A019E9A4203DD1D22A44B1A7080
:100CD0007FE40123039A137001F0A4F9FA23049A24
:100CE0009B005343039A0A3B1B18536085E4A300FF
:100CF000FF1A002320001A003900FFF7B3FB9A4EB9
:100D00009A4C3168200003F075FA3168200003F036
:100D1000B2FB3168200001F055FC914B1B78002B91
:100D200001D0019E55E42B68029A1C1213408A4A96
:100D30009B009B5804357DE4894BA4001B783F1B26
:100D4000002B01D0019E44E42B68029A1C12134030
:100D5000814A9B009B5804356CE4039803F0D2F859
:100D60007F4B1B78002B01D0019E32E42B68029A46
:100D70001C121340784A9B009B5804355AE43B1FD1
:100D80001868002824D1083B1868C30701D5401013
:100D900017E083070FD104280DD90F2302681340F1
:100DA000062B02D1FFF734FB0BE0052B03D1FFF735
:100DB0002FFB800005E01922694B019E1A70FFF796
:100DC00008FC3A0001214300083A0B43136001E09C
:100DD00040100138002832DD012243001343391F3F
:100DE0000B603B00083B1B681341181A3B000C3B8F
:100DF0001B68134203D08018A400904015E09907A7
:100E000017D1042B15D90F211E683140062906D1B0
:100E100001308000C358019AA400A35010E00529B6
:100E200007D118180079A4004000019B1043E0503E
:100E300006E019224A4B019E1A70FFF7CAFB0435DF
:100E4000474B1B78002B02D0019EFFF7C2FB2B689B
:100E5000029A1C121340404A9B009B580435FFF72E
:100E6000E9FBA300069AFB189B1ADB2B01DC01228D
:100E700005E01A223A4B019E1A70FFF7AAFB631E87
:100E8000002C03DD3A601C000437F8E7344B1B7874
:100E9000002B02D0019EFFF79CFB2B68029A1C12CC
:100EA00013402D4A9B009B580435FFF7C3FB069A5D
:100EB0003B1D9B1A2A4EDB2B04DD1A233370019E47
:100EC000FFF787FB019B069AA400934218D93B1FAA
:100ED0001868FFF78FFA002810DD019B0C3B1B6898
:100EE0005B1098420ADC9A07D31A1818204BC018D6
:100EF000019B8000C2583B1B1A6003E0202300E0E6
:100F000018233370164B3E1B1B78371D002B02D065
:100F1000019EFFF75EFB2B68029A1C1213400E4ADB
:100F20009B009B580435FFF785FBA3009C46F81AED
:100F3000002C04DC1C220A4B00261A7024E000213D
:100F400003685B1001268A008258164012D10D22D8
:100F5000034B1A7018E0C0467CA200009F86010077
:100F6000C802002080EE3600D0020020D40200200B
:100F7000FCFFFF3F5210934200DD130001318C4211
:100F8000E0DC01265B001E4363460660FE1AD34B7D
:100F9000371D1B78002B02D0019EFFF71AFB2B6830
:100FA000029A1C121340CE4A9B009B580435FFF74F
:100FB00041FBA3009C46F81A002C04DC1C22C74B02
:100FC00000261A7015E0002103685B1001268A00D4
:100FD0008258164003D10D22C04B1A7009E05210FE
:100FE000934200DA130001318C42EFDC01265B00F2
:100FF0001E4363460660FE1AB84B371D1B78002B54
:1010000002D0019EFFF7E5FA2B68029A1C121340EA
:10101000B34A9B009B580435FFF70CFB3B00083B91
:101020001868FFF7E7F93B1F04901868FFF7E2F92B
:10103000049AA600BC1B0023824200DA043323601A
:10104000A64BBE1B1B78371D002B02D0019EFFF75D
:10105000C0FA2B68029A1C121340A14A9B009B58AD
:101060000435FFF7E7FAA300FE1A04933B00083BA0
:101070001868FFF7BFF93B1F04001868FFF7BAF9BB
:10108000E20FC317A04253419B003360049BFE1A3A
:10109000924B371D1B78002B02D0019EFFF799FA67
:1010A0002B68029A1C1213408D4A9B009B580435F2
:1010B000FFF7C0FA3B00083B18683B1F1968A30004
:1010C000884202D1FB1A042222E004281ED9012200
:1010D000104201D0114219D10326304215D10F23FD
:1010E00002681A40042A10D131420ED104290CD9C9
:1010F0000A681340042B08D1FFF796F9431E984164
:10110000A600BE1B8000306003E0A3000022FB1A93
:101110001A60724BA4001B783E1B371D002B02D0B7
:10112000019EFFF756FA2B68029A1C1213406C4A74
:101130009B009B580435FFF77DFA3B00083B18687D
:101140003B1F1968A300884202D1FB1A002223E04A
:1011500004281FD90122104201D011421AD10326BE
:10116000304216D10F2302681A40042A11D13142AD
:101170000FD104290DD90A681340042B09D1FFF7B8
:1011800053F9030058425841A600BE1B800030604E
:1011900003E0A3000422FB1A1A60504BA4001B7842
:1011A0003E1B371D002B02D0019EFFF712FA2B6861
:1011B000029A1C1213404A4A9B009B580435FFF7C1
:1011C00039FAA300FE1A04933B00083B1868FFF7A6
:1011D00011F93B1F04001868FFF70CF9E217C30F61
:1011E000844253419B003360049BFE1A3B4B371DE6
:1011F0001B78002B02D0019EFFF7EBF92B68029AB7
:101200001C121340364A9B009B580435FFF712FA14
:101210003B00083B1868FFF7EDF83B1F0490186887
:10122000FFF7E8F8049AA600BC1B0023824200DD09
:1012300004332360294BBE1B1B78371D002B02D0C3
:10124000019EFFF7C6F92B68029A1C121340244A2C
:101250009B009B580435FFF7EDF93B1F1B68A4006A
:10126000043B591E8B413A1B9B0013601B4B171DFF
:101270001B78002B02D0019EFFF7ABF92B68029A76
:101280001C121340164A9B009B580435FFF7D2F9F5
:10129000A300FC1A04933B00083B1868FFF7AAF868
:1012A0003B1F06001868FFF7A5F836180120049BBD
:1012B000760006432660FE1A084B371D1B78002B6C
:1012C00002D0019EFFF785F92B68029A1C12134089
:1012D000034A9B009B580435FFF7ACF9C802002075
:1012E0007CA20000A300FE1A04933B00083B186890
:1012F000FFF780F83B1F04001868FFF77BF8241AFB
:101300000120049B640004433460FE1AEA4B371D3D
:101310001B78002B02D0019EFFF75BF92B68029A25
:101320001C121340E54A9B009B580435FFF782F9D5
:10133000A300FC1A04933B00083B1868FFF75AF817
:101340003B1F06001868FFF755F846430120049B31
:10135000760006432660FE1AD74B371D1B78002BFC
:1013600002D0019EFFF735F92B68029A1C12134038
:10137000D24A9B009B580435FFF75CF93B1F186865
:10138000FFF738F8A30006000493FC1A002803D1E5
:101390001F22C94B1A700AE03B00083B1868FFF790
:1013A00029F8310005F066FE012640000643049B43
:1013B0002660FE1AC04B371D1B78002B02D0019E01
:1013C000FFF707F92B68029A1C121340BB4A9B00D7
:1013D0009B580435FFF72EF93B1F1868FFF70AF8F2
:1013E000A30006000493FC1A002803D11F22B24B6D
:1013F0001A700AE03B00083B1868FEF7FBFF31005B
:1014000005F01EFF012649000E43049B2660FE1ACC
:10141000A94B371D1B78002B02D0019EFFF7D9F88E
:101420002B68029A1C121340A44A9B009B58043557
:10143000FFF700F93B1F1868FEF7DCFFC317C01861
:1014400058400123400018439B4BA4001B783E1BCF
:101450003060371D002B02D0019EFFF7BAF82B68D1
:10146000029A1C121340954A9B009B580435FFF7C3
:10147000E1F8A300FE1A07933068012C03D1FEF7B0
:10148000B9FF049008E0FEF7B5FF04007068FEF7AE
:10149000B1FF0130031B0493049B002B01DC0123EB
:1014A000049307F09BFF049905F0CAFE0C19012173
:1014B000079B64000C433460FE1A7F4B371D1B787A
:1014C000002B02D0019EFFF784F82B68029A1C12B1
:1014D00013407A4A9B009B580435FFF7ABF8A300F2
:1014E000FE1A31002000049300F0AAFF049B306034
:1014F000FE1A714B371D1B78002B02D0019EFFF79F
:1015000068F82B68029A1C1213406C4A9B009B5887
:101510000435FFF78FF8A300FE1A04933B00083B45
:101520001868FEF767FF3B1F04001868FEF762FFAC
:1015300004400120049B640004433460FE1A5E4BA7
:10154000371D1B78002B02D0019EFFF742F82B6855
:10155000029A1C121340594A9B009B580435FFF70E
:1015600069F8A300FC1A04933B00083B1868FEF7D7
:1015700041FF3B1F06001868FEF73CFF06430120B1
:10158000049B760006432660FE1A4B4B371D1B78E2
:10159000002B02D0019EFFF71CF82B68029A1C1248
:1015A0001340464A9B009B580435FFF743F8A300BD
:1015B000FC1A04933B00083B1868FEF71BFF3B1F17
:1015C00006001868FEF716FF46400120049B7600CF
:1015D00006432660FE1A384B371D1B78002B02D0BD
:1015E000019EFEF7F6FF2B68029A1C121340334A45
:1015F0009B009B580435FFF71DF83B1F1868FEF74A
:10160000F9FEC0430123400018432B4BA4001B7874
:101610003E1B3060371D002B02D0019EFEF7D9FF24
:101620002B68029A1C121340244A9B009B580435D5
:10163000FFF700F8A300FE1A04933B00083B18686C
:10164000FEF7D8FE3B1F04001868FEF7D3FE844067
:10165000012364001C43049B3460FE1A164B371DA3
:101660001B78002B02D0019EFEF7B3FF2B68029A75
:101670001C121340114A9B009B580435FEF7DAFFF9
:10168000A300FE1A04933B00083B1868FEF7B2FE65
:101690003B1F04001868FEF7ADFE044101236400FF
:1016A0001C43049B3460FE1A034B371D1B78002B30
:1016B00006D0019EFEF78DFFC80200207CA200002C
:1016C0002B68029A1C121340E94A9B009B58043570
:1016D000FEF7B0FF3B000C3B1868FEF78BFE3B00AB
:1016E000083B06001868FEF785FEF1170200C317D5
:1016F000300005F0F7FD3B1F049005911868FEF7D8
:1017000079FE02000498059905F0A0FD0123400030
:101710001843D84BA4001B783E1B3060371D002BAC
:1017200002D0019EFEF755FF2B68029A1C1213404F
:10173000CF4A9B009B580435FEF77CFFA300FE1A9E
:10174000310020000493FEF772FD049B3060FE1A06
:10175000C84B371D1B78002B02D0019EFEF739FFC6
:101760002B68029A1C121340C14A9B009B580435F7
:10177000FEF760FFA300FE1A310020000493FEF77D
:1017800066FD049B3060FE1ABA4B371D1B78002B98
:1017900002D0019EFEF71DFF2B68029A1C12134017
:1017A000B34A9B009B580435FEF744FFA300FF1A81
:1017B00039002000FEF75DFDAE4B1B78002B02D0F8
:1017C000019EFEF706FF2B68029A1C121340A84ADE
:1017D0009B009B580435FEF72DFFA300FE1A310035
:1017E00020000493FEF777FD049B3060FE1AA14BA6
:1017F000371D1B78002B02D0019EFEF7EAFE2B68F6
:10180000029A1C1213409A4A9B009B580435FEF71B
:1018100011FFA300FF1A39002000FEF792FD954B3F
:101820001B78002B02D0019EFEF7D3FE2B68029A94
:101830001C1213408E4A9B009B580435FEF7FAFE9B
:10184000A300FE1A310020000493FEF7B3FD049BB1
:101850003060FE1A874B371D1B78002B02D0019E8B
:10186000FEF7B7FE2B68029A1C121340804A9B00B9
:101870009B580435FEF7DEFE069A3B1D04937D4C13
:101880009B1ADB2B04DD1A23019E2370FEF7A1FEB9
:1018900000F0D2FB01234000184323783860002B6E
:1018A00003D0019E049FFEF794FE2B68029A1C123F
:1018B00013406F4A9B009B58049F0435FEF7BAFE05
:1018C000069A3B1D04936B4C9B1ADB2B04DD1A23F9
:1018D000019E2370FEF77DFE00F0A4FB664B4000E6
:1018E00018400123184323783860002B03D0019E51
:1018F000049FFEF76EFE2B68029A1C1213405C4A8E
:101900009B009B58049F0435FEF794FEA300FB1A2E
:101910000493012320001A000499FEF7A3FD574CFD
:101920002068643002F08AFA002816D0039B2168F0
:101930005A78534802F0ADFD15E0A300FB1A04935A
:101940002000012300220499FEF78CFD4B4C2068F7
:10195000643002F073FA002802D1043DFEF74DFE18
:10196000474802F0A5FB0123039A137000F05AFBCD
:10197000444A23681268063353431818039B58607F
:10198000FEF73CFEFEF7E6FD3A4BA4001B783E1B3B
:101990003060371D002B02D0019EFEF71AFE2B6827
:1019A000029A1C121340324A9B009B580435FEF7E2
:1019B00041FEA4003E1B300000F074FB2D4B306054
:1019C0001B78371D002B02D0019EFEF702FE2B680C
:1019D000029A1C121340264A9B009B580435FEF7BE
:1019E00029FEA4003E1B300000F05EFB214B30605E
:1019F0001B78371D002B02D0019EFEF7EAFD2B68F5
:101A0000029A1C1213401A4A9B009B580435FEF799
:101A100011FEA4003E1B300000F048FB154B306067
:101A20001B78371D002B02D0019EFEF7D2FD2B68DC
:101A3000029A1C1213400E4A9B009B580435FEF775
:101A4000F9FDA4003F1B380000F04EFB094B1B784A
:101A5000002B02D0019EFEF7BCFD2B68029A1C12DF
:101A60001340034A9B009B580435FEF7E3FDC04634
:101A70007CA20000C8020020FEFFFF7FD0020020F1
:101A8000D402002004000020A300FE1A3100200030
:101A9000049300F04BFB049B3060FE1AE64B371DAD
:101AA0001B78002B02D0019EFEF793FD2B68029A53
:101AB0001C121340E14A9B009B580435FEF7BAFD07
:101AC000A4003F1B380000F06BFBDB4B1B78002BA6
:101AD00002D0019EFEF77DFD2B68029A1C12134076
:101AE000D64A9B009B580435FEF7A4FD0121200037
:101AF00000F03EFBD04B1B78002B02D0019EFEF77E
:101B000068FD2B68029A1C121340CC4A9B009B581C
:101B10000435FEF78FFD0021200000F029FBC64BA5
:101B20001B78002B02D0019EFEF753FD2B68029A12
:101B30001C121340C14A9B009B580435FEF77AFDE6
:101B4000A4003E1B300000F049FBBB4B30601B780B
:101B5000371D002B02D0019EFEF73BFD2B68029A39
:101B60001C121340B54A9B009B580435FEF762FDDA
:101B7000A4003E1B300000F045FBAF4B30601B78EB
:101B8000371D002B02D0019EFEF723FD2B68029A21
:101B90001C121340A94A9B009B580435FEF74AFDCE
:101BA000A4003F1B380000F007FBA34B1B78002B61
:101BB00002D0019EFEF70DFD2B68029A1C12134005
:101BC0009E4A9B009B580435FEF734FDA4003F1B42
:101BD000380002F00FFF984B1B78002B02D0019EBB
:101BE000FEF7F7FC2B68029A1C121340934A9B00E5
:101BF0009B580435FEF71EFDA4003E1B300002F08A
:101C00008DFF8D4B30601B78371D002B02D0019E5D
:101C1000FEF7DFFC2B68029A1C121340874A9B00D8
:101C20009B580435FEF706FDA4003F1B380002F068
:101C300091FE814B1B78002B02D0019EFEF7C9FC60
:101C40002B68029A1C1213407C4A9B009B58043557
:101C5000FEF7F0FCA4003E1B300002F091FE764B34
:101C600030601B78371D002B02D0019EFEF7B1FCBF
:101C70002B68029A1C121340704A9B009B58043533
:101C8000FEF7D8FCA300FF1A3900200000F008FF7F
:101C9000694B1B78002B02D0019EFEF79AFC2B6843
:101CA000029A1C121340654A9B009B580435FEF7AC
:101CB000C1FCA300FF1A3900200000F07BFD5E4B41
:101CC0001B78002B02D0019EFEF783FC2B68029A42
:101CD0001C121340594A9B009B580435FEF7AAFC7E
:101CE000A300FF1A3900200000F074FD524B1B784E
:101CF000002B02D0019EFEF76CFC2B68029A1C128E
:101D000013404E4A9B009B580435FEF793FCA300FA
:101D1000FF1A3900200000F085FD474B1B78002B8F
:101D200002D0019EFEF755FC2B68029A1C1213404C
:101D3000424A9B009B580435FEF77CFCA300FE1A28
:101D400031002000049302F073FF049B3060FE1A00
:101D5000394B371D1B78002B02D0019EFEF739FC52
:101D60002B68029A1C121340344A9B009B5804357E
:101D7000FEF760FCA300FE1A31002000049302F07D
:101D80005FFF049B3060FE1A2B4B371D1B78002B26
:101D900002D0019EFEF71DFC2B68029A1C12134014
:101DA000264A9B009B580435FEF744FCA300FE1A0C
:101DB00031002000049302F04BFF049B3060FE1AB8
:101DC0001D4B371D1B78002B02D0019EFEF701FC36
:101DD0002B68029A1C121340184A9B009B5804352A
:101DE000FEF728FCA300FE1A31002000049302F045
:101DF00069FD049B3060FE1A0F4B371D1B78002BCA
:101E000002D0019EFEF7E5FB2B68029A1C121340DC
:101E10000A4A9B009B580435FEF70CFCA300FF1AEE
:101E20003900200000F0DAFD034B1B78002B07D0AF
:101E3000019EFEF7CEFBC046C80200207CA2000037
:101E40002B68029A1C121340414A9B009B58043590
:101E5000FEF7F0FBA300FF1A3900200000F00AFD96
:101E60003C4B1B78002B02D0019EFEF7B2FB2B6887
:101E7000029A1C121340364A9B009B580435FEF709
:101E8000D9FBA300FE1A31002000049300F01EFECF
:101E9000049B3060FE1A2F4B371D1B78002B02D09D
:101EA000019EFEF796FB2B68029A1C121340284AEB
:101EB0009B009B580435FEF7BDFBA300FF1A3900B9
:101EC000200000F073FD234B1B78002B02D0019EF5
:101ED000FEF77FFB2B68029A1C1213401C4A9B00E2
:101EE0009B580435FEF7A6FBA300FF1A390020001B
:101EF00001F026FF174B1B78002B02D0019EFEF746
:101F000068FB2B68029A1C121340114A9B009B58D5
:101F10000435FEF78FFBA300FE1A31002000049366
:101F200001F00EFF049B3060FE1A0A4B371D1B7830
:101F3000002B02D0019EFEF74CFB2B68029A1C126C
:101F40001340034A9B009B580435FEF773FBC046C1
:101F50007CA20000C80200200023F7B55A1E01929F
:101F6000002B07DA00F0E6FD02F090F902F0B6FA75
:101F70006423019300263000194B19688E4201DB5F
:101F8000019BEBE7174B1A680132914200DC0022FB
:101F9000F0241A601D68144F6C43E35D002B1DD0C4
:101FA000E419022B16D0012B0ED1002801D100F02C
:101FB00039F8F0226A430C4B0C499B185B68C31A32
:101FC0008B4201D80223BB54F0235D43064BEB5CEC
:101FD000022B03D12000FEF7D5FAD1E70136CBE77B
:101FE000CC020020000000207C1200209F8601000F
:101FF0000020704700207047002070470020704785
:1020000001220020054B06491A6158500330043163
:1020100058508018083158501A60704700800040AE
:10202000040500000122034B1A64A822D20098582C
:102030007047C0460080004010B5FFF7F3FFFA215B
:10204000890004F08DFF10BD10B50100014804F0B7
:10205000F7FA10BD041200200048704784A4000065
:102060001D20704770B5054E0400335C0D008B4297
:1020700002D004F0EFFE355570BDC04618060020B2
:1020800070B50024064D635D012B05D100212000B1
:1020900004F0E0FE0023635501341D2CF2D170BD25
:1020A000180600200D2070473B207047036870B56C
:1020B0005B100120052B12D8094A9B009C58094D42
:1020C0002B5D002B05D00021200004F0C3FE00236F
:1020D0002B55200004F068FD01234000184370BD1B
:1020E000B4A400001806002070B5036845685C10B1
:1020F0006D1004D40B4B9D4202DD1D0000E0002555
:102100001C2C0DD8084E335D012B05D00121200079
:1021100004F0A0FE012333552900200004F0D2FD75
:1021200070BDC046FF030000180600200B6870B5A4
:102130005D101C2D16D80024012804DD4C68043CD9
:10214000624262415400094E735D9C4204D02100FA
:10215000280004F07FFE7455280004F0AFFE04232D
:10216000012800D00023180070BDC04618060020CA
:1021700070B504000D001C280ED8084E335C012BEE
:1021800004D0012104F066FE01233355290020000C
:102190004D1EA94104F07CFE70BDC046180600200B
:1021A000436810B5191F4A424A41006811004010A7
:1021B000FFF7DEFF10BD000037B56A46064B6946E3
:1021C00030CB30C203680220042B02D100F002FBA6
:1021D00001E000F027FB37BD7CA4000010B5084CDF
:1021E0006379002B05D00021052004F033FE002385
:1021F0006371052004F062FE43425841800010BD27
:102200001806002010B5084CE37A002B05D00021F9
:102210000B2004F01FFE0023E3720B2004F04EFE9F
:1022200043425841800010BD180600207047704797
:1022300010B5034A0421034801F06EFD10BDC046ED
:102240000800002070AB0000E12110B549020948E8
:1022500004F0D4FAFFF7D4FE0A2004F09FFC002318
:10226000FF21054A995401331D2BFBD100F0B6FD27
:1022700010BDC0460412002018060020F8B50B4E11
:10228000070030000D0004F0F9FA041EAC4200DD36
:102290002C003D00EB1B9C4205DD300004F0F8FAF9
:1022A00028700135F6E72000F8BDC0460412002072
:1022B00010B50100014804F0A9FA10BD0412002075
:1022C00010B5054C200004F0AFFAE12120004902CE
:1022D00004F094FA10BDC04604120020064B012001
:1022E0001A68064B06491A60C82200235200C850DB
:1022F00004339342FBD1704740060020380600208B
:10230000D423002000B59BB00200054901A807F0C6
:10231000E5F801A801F0E8FE02F0E0F8FCE7C046AD
:10232000CCA4000037B5184D04002868002801D05F
:1023300006F0C8FCA400200006F0BAFC28600028C3
:1023400001D1124809E001AB984208D2104B0219A2
:102350006B440193934202D20E48FFF7D3FF042847
:1023600002D808302860083C2B680B4A1C191360FF
:102370000A4BC8221C600120002309495200C850A2
:1023800004339342FBD137BD40060020DDA400009A
:102390001CFCFFFF0DA50000380600203C060020B5
:1023A000D423002070B50D4D0D4E2B684C1CA4009D
:1023B00036681C19B44203D90A20FEF7C5F80BE0B1
:1023C0002C601D00AC4201D904C5FBE70F220901B6
:1023D000104008431860180070BDC0463806002041
:1023E0003C0600200322CB1C70B50C00D91711400D
:1023F000C9180500891000220420FFF7D3FF00232D
:10240000A34204DAE95CC21811710133F8E7E14331
:102410000023C917214041180B7170BD10B5830707
:1024200006D1042804D90F2304C81340042B03D079
:102430000E20FEF789F8014810BDC046A6AA00008C
:1024400010B503240868044006D1042804D90F23DA
:1024500002681340042B01D00E2011E0FFF7DEFFCD
:102460000378233B5942594110224018210007F0BC
:1024700015F980239B05C218054B9A4203D91420F5
:10248000FEF762F802E001234000184310BDC04689
:10249000FFFFFF3F70B501240B680D001C4001D009
:1024A0005C1002E00D20FEF74FF8200005F05AF80E
:1024B000264904F043FF06F01DFB02F02FFF002227
:1024C000234B05F0D1FC0023002204F001FF01247E
:1024D0002B681C40002819D0002C01D05C1002E0B1
:1024E0000D20FEF731F8200005F03CF8174904F004
:1024F00025FF06F0FFFA02F011FF0022144B05F051
:10250000B3FC0022134B05F075F818E0002C01D045
:102510005C1002E00D20FEF717F8200005F022F80D
:102520000A4904F00BFF06F0E5FA02F0F7FE00227C
:10253000074B05F099FC0022064B05F00FFF06F053
:1025400061FA01234000184370BDC046D3023739F9
:102550000000D0400000E03F10B5034A02210348CC
:1025600001F0DAFB10BDC0462800002078A500006D
:102570000020704710B51E20FDF7E6FF10BD10B516
:102580001E20FDF7E1FF10BD10B51E20FDF7DCFF9A
:1025900010BD10B51E20FDF7D7FF10BD10B51E20D1
:1025A000FDF7D2FF10BD10B51E20FDF7CDFF10BD09
:1025B00010B51E20FDF7C8FF10BD10B51E20FDF799
:1025C000C3FF10BD7047000010B5034A092103483E
:1025D00001F0A2FB10BDC046380000208AA5000013
:1025E0000123034A1360034A106898401843704758
:1025F0004C06002054060020F0B5EFF310810123B3
:10260000194083F31088134E134AB4461268013AF6
:102610009340124A1468124A1568124A002B15D0CA
:10262000166803420BD02660C046C046C046C0466E
:10263000C046C046C046C04616682E6004E06746E5
:102640003E601668084F3E605B08E7E781F310883C
:10265000F0BDC04608050050C800002060060020FC
:102660005C060020480600200C05005030B585B0FF
:1026700001AD0C220649280006F02EFB0024285D3F
:1026800001210134FFF7EEFC0C2CF8D105B030BD70
:1026900016A60000F0B53B4C85B0210003220C319A
:1026A000684606F019FB210001AE0F310922300007
:1026B00006F012FBFFF7C0FC334B344CC018236804
:1026C000984201D2002323602568002D3CD1775D1C
:1026D00001213800FFF7C6FC01350121380004F064
:1026E000D7FB092DF3D100256B465E5D012130003B
:1026F000FFF7B8FC01350021300004F0C9FB032DC1
:10270000F2D1C82080000138C046C046C046C0464D
:10271000C046C046C046C046C046C046C046C04689
:10272000F1D100210420FFF79DFC00256B4600211C
:10273000585D0135FFF796FC032DF7D1FFF77CFCC0
:1027400013302060002519E0FFF776FC2368002590
:10275000984213D3042004F027FA0D4B0D4EC018F5
:1027600001D4306000E035603068032104F082FC61
:1027700000230125084A306023601360280005B05B
:10278000F0BDC04616A60000102700004406002039
:10279000C8FEFFFF540600204C06002010B501249F
:1027A000044001D0441002E00D20FDF7CDFE2000D2
:1027B00010BD00000022054B10B51A60044B1B68C9
:1027C000934201D002F0A6FA002010BD5806002066
:1027D0002811002070B508680D00FFF7DFFF040026
:1027E0006868FFF7DBFF631E0100042B14D8451E49
:1027F000042D11D805226A43D318012215009D40EB
:102800002B00064805682B430360054B1B68002B13
:1028100002D0200002F07FFA002070BD5806002090
:102820002811002070B508680D00FFF7B7FF0400FD
:102830006868FFF7B3FF631E0100042B14D8451E20
:10284000042D11D805226A43D31801229A4013009F
:10285000064802689A43064B02601B68002B03D0AF
:102860000022200002F057FA002070BD5806002018
:1028700028110020F0B5050085B008680C00FFF7AE
:102880008DFF0390022D08DD6068FFF787FF0700CA
:10289000A068FFF783FF040001E00124270005235F
:1028A0006343053B0293012326000193231D9E42AF
:1028B00034DC3D003B1D9D422BDC731E042B23D8D2
:1028C0006B1E042B20D8029B039A591E019B4919A9
:1028D0001A40204B0AD001228A4019680A431A6024
:1028E0001D4B01221B68002B0ED009E001208840FF
:1028F0000100186888431860174B1B68002B03D031
:102900003100280002F007FA019B01355B000193BA
:10291000D0E7029B013605330293C7E73D1D042D26
:1029200015D8012C13D126003300AB40094A116899
:102930009943094B11601B68002B04D0781D0022BD
:10294000210002F0E8F901340535062CECD1002015
:1029500005B0F0BD580600202811002010B5041E57
:1029600013DBFFF77DFB84420FDA094BA400E2582A
:1029700001239340074A08491360084A1160084A36
:1029800008491160084A136010BD0024EDE7C046F5
:1029900000AE000048060020080500506006002038
:1029A0005C0600200C050050180500500B6810B59F
:1029B0000200D80701D5581001E001204042182339
:1029C000012A03DD4A68042A00D10833024A136051
:1029D000FFF7C4FF002010BDC80000202D4BF7B545
:1029E0001B680C00002B03D101204042FFF7B6FF0B
:1029F00001262468344219D0FF2263101802120401
:102A00001040FF22611212020A40DBB21043184349
:102A1000214B1B68202B06D1B440204BA40EA400F0
:102A2000E35800021843FFF7E7FD30E00325254097
:102A30002DD1042C2BD90F2322681340062B26D12D
:102A4000FF27130901933F04019B9D421FDAAB004E
:102A5000E3185A68324218D0531018023840FF2148
:102A600084460902501208406146DBB2084318430D
:102A7000094B1B68202B06D15200920E074B920087
:102A8000D35800021843FFF7B7FD0135DCE70020FB
:102A9000FEBDC04648060020C8000020A4A60000D5
:102AA000086810B5C30703D5FFF778FE054B18601B
:102AB000054B1B68002B03D0024B186802F02CF961
:102AC000002010BD58060020281100200868F8B525
:102AD000C30702D5FFF762FE0BE0830726D1042867
:102AE00024D90F2203681A40042A1FD11B091DD0C4
:102AF00000790300203B5E2B18D8052200205343A9
:102B00000B4E9D18043AAB420CD0052110249F5D5A
:102B10003C4200D080180139520064100029F7D1DE
:102B20000133F0E701234000184300E00120F8BD25
:102B3000A4A700007FB5A44E3368002B0BD1A34A95
:102B40001268002A07D1A24B1B68002B00D139E183
:102B5000FFF7A0FD36E19F4D2A68002A2AD19C4A42
:102B60001268002A07D0FFF795FD002800D129E15F
:102B7000FFF77CFD05E0954A1268002A01D1002B81
:102B8000F6D1924B19681A00002911D03468002C34
:102B90000ED101AD0C22904928001C6006F09CF873
:102BA000285D00210134FFF75DFA0C2CF8D109E112
:102BB0003368136000211A2004F06AF900211B20F9
:102BC00004F066F900211C2004F062F92E68012E41
:102BD00056D0022E00D19CE0002E00D0ECE0013651
:102BE00031007A4C03202368994304F051F9042002
:102BF000216801400B005942594104F049F9102164
:102C000023680A200B405942594104F041F98021C0
:102C1000236809010B4059425941062004F038F954
:102C20008021236809020B4059425941072004F0D2
:102C30002FF98021236849020B405942594109204C
:102C400004F026F98021236889020B40594259413A
:102C5000192004F01DF980212368C9020B40594254
:102C60005941182004F014F9802321681B030B40FC
:102C700059425941172004F00BF931001A2099E00C
:102C80000221524C172023680B405942594104F04D
:102C9000FFF80821236818200B405942594104F0DD
:102CA000F7F880212368C9000B405942594104209C
:102CB00004F0EEF88021236849010B405942594144
:102CC0000A2004F0E5F880212368C9010B4059422D
:102CD0005941032004F0DCF88021236889030B406C
:102CE00059425941092004F0D3F8802321681B047C
:102CF0000B4059425941192004F0CAF8310006200E
:102D000004F0C6F83100072004F0C2F831001B209F
:102D100050E020212D4C172023680B405942594187
:102D200004F0B6F84021236818200B40594259415D
:102D300004F0AEF88021236819200B405942594114
:102D400004F0A6F88021236849000B4059425941FC
:102D5000092004F09DF88021236889000B40594226
:102D60005941072004F094F88021236889010B4021
:102D700059425941062004F08BF880212368490309
:102D80000B40594259410A2004F082F880212368FF
:102D9000C9030B4059425941032004F079F88023BC
:102DA00021685B040B4059425941042004F070F83B
:102DB00001211C2004F06CF82B680321581C04F03E
:102DC0003FFA29607FBDC04658060020500600200B
:102DD0004C0600206406002016A60000012010B555
:102DE0004042FFF7BBFD10BD10B5034A092103485F
:102DF00000F092FF10BDC046800000202EA600000B
:102E000030B502248025094B094AED009C505C59DD
:102E1000002CFCD0A124E400884204D28025ED00DF
:102E200018514019F8E70021995030BD00E00140E9
:102E30000405000010B5002804D1C020B0214002D4
:102E4000890203E0B02080218002C902FFF7D8FF89
:102E500010BD002802D0B0239B0201E0C0235B021A
:102E60001B6800201A0E532A01D11B02180A704752
:102E700030B501248025064A064BED00D450545944
:102E8000002CFCD001600021014AD15030BDC04669
:102E900000E001400405000010B5002802D0B02079
:102EA000800201E0C0204002A6230902DB05090AD6
:102EB0001943FFF7DDFF10BDF0B5012480250300A5
:102EC0000F4F08000F49ED007C507C59002CFCD0BE
:102ED0009C46002810DD54781678937824023443F9
:102EE0001B0423431C00D37801381B06234364468C
:102EF00008C40432A446ECE700237B50F0BDC04672
:102F000000E001400405000070B505004B680A00B0
:102F10009C1C2100FFF7D0FFA000281870BD000006
:102F2000154B1B68002B04D08021B023C9029B02E3
:102F300003E0B021C02389025B02002807D1191DDC
:102F40005B6802001B0E522B14D10A0012E0002213
:102F500081420FD903681B0E522B0BD143680233F9
:102F60009B00C318994205D91A68110E00225229F4
:102F700000D11A00100070476808002070B50020CA
:102F8000FFF7CEFFFF260500002808D003681C14B9
:102F90003440FFF7C5FFDA2CF6D10500F4E728002E
:102FA00070BD00008022F0B55200A1B0002165483C
:102FB00005F09BFE802200215200634805F095FE3B
:102FC000624C23681A00039353425A411000049242
:102FD000FFF730FF039B0594002B01D15C4C00E010
:102FE0005C4C0020FFF7CAFFFF270500002D7CD0B6
:102FF0002A68131412123A403B4002921A000A3A0D
:10300000092A42D84F4B029A995C002968D11022B4
:10301000514805F06AFE2E00336802991A123A40B0
:10302000914217D11A143A400B2A06D0132A0CD019
:103030000A2A0FD1484B1E600CE03B40022B09DCF2
:10304000454A9B00D3185E6004E0102200214248EC
:1030500005F04BFE3000FFF763FF061EDCD13E4B50
:10306000196800290FD02000FFF74EFF04003B4EE7
:103070003168002903D02000FFF746FF0400384BD9
:103080000436B342F4D12F4B27E01A00153A082A30
:1030900026D82D4A0299565C002E21D1152B00D13D
:1030A0002E00280003681A143A40152A03D01D2A5E
:1030B00007D1002605E0029A1B123B409A4200D13C
:1030C0000600FFF72DFF0028ECD1002E04D02000D1
:1030D0003100FFF719FF04001B4B0121029A99549C
:1030E0002800FFF71DFF050080E70398FFF7B1FEFA
:1030F000411C0498FFF7D0FE059B1A4D049A2C60E2
:103100001A60FFF7DDF8059B2C681B68002B02D0C6
:10311000B0239B0201E0C0235B026420A021E41ADB
:103120006043490203F0A6FFA0225202030000926E
:103130000D49220007A806F0D1F907A800F0D4FF36
:1031400021B0F0BD68070020680600206808002054
:1031500004C00200048001006425002068250020CE
:10316000742500206C0800208CA90000F0B5002018
:10317000B7B00024FFF7D4FE270005002600002D7D
:1031800020D0FF226B6828689C460233FF18031288
:103190000136134011009C4200DA1C0002140A4060
:1031A00003926246014001920091039A1C4904A8CF
:1031B00006F094F904A800F097FF2800FFF7B0FE8E
:1031C0000500DCE7174D2868FFF743FE3B00019040
:1031D00000943200144904A806F080F904A800F015
:1031E00083FF124B1C682B68002B02D0B0239B027C
:1031F00001E0C0235B026420A021E41A604349027D
:1032000003F038FFA0225202030000920849220076
:1032100004A806F063F904A800F066FF37B0F0BD1B
:10322000C2A9000068080020D6A900006C08002090
:10323000A7A9000070B50020FFF70BFE04000120D5
:10324000FFF707FE844200DA04000A4B1E6875424D
:10325000754128001D60FFF7EDFD002E01D0064BE3
:1032600000E0064B064A2800611C1360FFF714FEBD
:1032700070BDC046680800200480010004C0020040
:103280006C080020F8B50020FFF7E3FD07000120DF
:10329000FFF7DFFD3E00224D0643224C0CD180217A
:1032A000C020C9024002FFF7ABFD01213000FFF74B
:1032B000F3FD2E601C4B2FE0874208DD0023B02178
:1032C0002B60194B890223602368002011E0012341
:1032D00080212B60154BC9022360F5E71A68551C45
:1032E00018D0120E522A07D101205A6802329200D9
:1032F0009B188B42F2D311E0002800D023600C4CC5
:103300000C49200006F016F92000FEF79DFEFFF79D
:1033100091FF04E0002802D0236000E02160F8BDA6
:10332000680800206C0800200480010004C002002E
:10333000B02500200BAA0000F0B585B0039203224F
:103340000333DC1714402A4EE3189C1033680190B5
:103350000291002B02D08022D20201E0B022920220
:10336000244FA51C3B68AD005B199A4217D2FFF7AA
:1033700019FE3368002B02D08022D20201E0B02275
:1033800092023B685B199A4209D21B4C1B492000F0
:1033900006F0D0F82000FEF757FE002026E0029B42
:1033A0003E681B06190C6B461A7BA423DB051343EE
:1033B000019A0B431104FF221204114019433000FB
:1033C000FFF756FD3300301D0833210001933B60A9
:1033D000FFF74EFD002C04D00A9A21000198FFF758
:1033E0006BFD3000019B083D5D193D6005B0F0BDEF
:1033F000680800206C080020B025002034AA0000D6
:1034000010B5FFF7CFFD10BD70B59AB0FFF73AFFCA
:10341000FF22264CD2000021200005F066FC00208F
:10342000FEF7DCFE042804D10020FEF7EBFE0428A2
:1034300031D00020FFF7A2FDFF25002600281AD07A
:1034400003681A142A400A2A08D11A122A40FF2AAD
:103450000ED0D200A1180B71A05009E0132A07D199
:103460001B122B40FF2B03D0DB00E2181671E65035
:10347000FFF756FDE2E7FF210200C900235808309C
:103480005D1EAB41D2188842F8D1094901A806F067
:1034900025F801A802E0FFF7CDFE064800F024FE63
:1034A000054800F021FE1AB070BDC046DC1B0020AC
:1034B0005BAA000077AA00006FAA00000022012189
:1034C000094B5A60094A51605A68002AFCD0002210
:1034D000C021054B49001A61044B01329A60044B2C
:1034E00001325A501A607047FC1000400010004032
:1034F00000E100E00222064B0121DA670022054BC1
:103500005A61054A11615A69002AFCD07047C046C9
:1035100004E100E0FC1000400010004010B5054B35
:103520001A781C00002A01D0FFF7E4FF0020207069
:1035300010BDC046F8080020024B18680123400067
:1035400018437047F4080020004870478C2500207D
:10355000024B186801234000184370473C010020CB
:1035600070B504000D001600FEF766FD80230122F1
:1035700000215B055B6E6270E270020AA271020CB0
:10358000E2711A0A60716372000EA2721A0C1B0EAD
:1035900026702571A1702072E272237370BD000045
:1035A000124B10B51B68124C5A1C0FD0114C002B3B
:1035B0000CD0114C012B09D0104C022B06D00D4C15
:1035C000042B03D00E4C052B00D10B4C21000D48D1
:1035D00005F0B0FF200005F0B5FF0300042204331E
:1035E0009B0809481B011343036010BD40010020E4
:1035F00049AB000042AB000054AB000059AB0000E7
:103600004EAB0000782500207425002070B5214CB9
:103610002278002A3DD1204B01215A608022D20518
:1036200011605A68002AFCD0002207201B4B1C495D
:1036300001255A500439585008315A5019481A492E
:1036400058501A491A485A501A495A50A622D200BC
:103650009D50082218495A500431585002201749E9
:1036600058501748174958501748043958501820CF
:1036700016495850C12189005A500539FF395A5806
:10368000083802435A50124A12499950FFF716FF60
:10369000257070BDF8080020FC00004000100040BC
:1036A0000C050000746962751C050000240500000B
:1036B000200004022C050000140500003405000061
:1036C000FFFF00003C050000211001005405000030
:1036D000040500007008002010B500280EDD0C68FD
:1036E000E3070BD56410FF2C08D8054B1B78002B83
:1036F00001D1FFF78BFF034B034AD450002010BDCC
:10370000F8080020240500000010004013B5002830
:1037100015DD0C68E30712D508220A4968466410D3
:1037200005F0DAFA072C0AD8074B1B78002B01D1D9
:10373000FFF76CFF6B46054A1957054BD150002027
:1037400016BDC0463AAB0000F8080020001000404B
:103750000C05000010B5002813DD0C68E30710D538
:103760006410532C0DD8084B1B78002B01D1FFF7A8
:103770004DFFFFF7BFFEA123044ADB00D450FFF743
:103780009DFE002010BDC046F8080020001000403B
:1037900070B50E4B06001B78002B01D1FFF736FFEA
:1037A00000200B4D2C7884420ED00A4B2022197831
:1037B0000323091B1940084B49015918300005F033
:1037C0008BFA0120013C2C7070BDC046F808002027
:1037D000F9080020F008002070080020002330B510
:1037E00089B0984226DD03240D682C409C4221D1EB
:1037F0002300042D1ED90F212A681140062919D152
:1038000012091F2A16D96846FFF7C2FF23000028B5
:1038100010D06B46012019780123A14203DB6B46CF
:103820001B5D5B000343A200AA1801345360202CE7
:10383000F2D10423180009B030BD0000F0B5434BAD
:103840008BB01B78002B01D1FFF7E0FE02AD280002
:10385000FFF79EFF002873D02B780B2B70DD6B7861
:10386000012B6DD1EA780023012A69D1384F394CF8
:103870003B6023712B79384A1360002B0ED115253C
:103880006D446A782878AB78120202431B04134314
:103890001A00EB781B0613433B6053E0012B11D158
:1038A00015266E4472783078B378120202431B04F6
:1038B00013431A00F3781A261B0613433B606A7CF5
:1038C0000E2327E0022B03D16A7B1033162621E05A
:1038D000042B0DD1152108226944684605F0FCF936
:1038E0000098019901F078FC05F08CF8386029E027
:1038F000052B27D1152108226944684605F0ECF90B
:103900000098019901F068FC05F07CF81E260A2356
:1039100038606A7D6E44934200DB130000229342BC
:1039200004D0B05CA11808710132F8E7042000212E
:10393000E21804339B101B0103431171236003E061
:10394000002001E00022E8E70BB0F0BDF8080020FD
:10395000F40800208C2500204001002010B5041E32
:1039600026D0144B1B78002B01D1FFF74FFEFFF739
:10397000C1FD00201049114A114B8C505860013094
:10398000086059680029FCD000200D4908610A49E7
:103990000130886019690029FCD00A4B0A491B785C
:1039A0005B01CB1804498B50FFF7A4FDFFF786FDA0
:1039B00010BDC046F80800200010004004050000BB
:1039C000FC100040F00800207008002030B589B0DD
:1039D00000281EDD03230A6813401AD1042A18D9CF
:1039E0000F2011680840062813D109091F2910D992
:1039F00001240133990051580020214201D049107F
:103A0000C8B26D46591E6854202BF2D16846FFF7A4
:103A1000A5FF002009B030BD30B589B0002826DDF3
:103A20000868830723D1042821D90F230268134093
:103A3000042B1CD1FEF7F2FC050005F083FD041EEB
:103A4000122C00DD1224220002210D326846FFF7FD
:103A500087FD6B465C730023A34205DA1A00E95C1C
:103A60006A4491730133F7E76846FFF777FF002058
:103A700009B030BD70B50C0088B0012833DD08688E
:103A8000830730D104282ED90F2302681340042B5A
:103A900029D14B68DB0726D5FEF7C0FC060005F0F0
:103AA00051FD6468050064100E2800DD0E252A0013
:103AB000012111326846FFF753FD6B466A465C737D
:103AC000231293732314D3730023240E1474557498
:103AD000AB4205DA1A00F15C6A4491740133F7E7EE
:103AE0006846FFF73BFF002008B070BD30B589B0D5
:103AF000002814DD0C68E30711D510226846002168
:103B0000FFF72EFD6B466A4665105D7368466312CB
:103B10002D0E64149373D4731574FFF71FFF0020E8
:103B200009B030BD184B10B55A681849002A03D0A7
:103B300000225A6001328A601B691448002B22D08F
:103B40000023114A13618022D2008458104A012CAC
:103B500016D1A923DB00C3585B4213600D4A1378CA
:103B6000032B01D80133137003220B480378013370
:103B700013400A4A03705B01D318094A8B5000E0D6
:103B8000136001238B6010BDFC100040001000404A
:103B90003C010020F9080020F008002070080020F7
:103BA0000405000010B5034A0E21034800F0B4F8E4
:103BB00010BDC046CC00002060AB0000044A05499F
:103BC0001368C85401339B059B0D13607047C046B2
:103BD000040D0020FA080020114A70B51368114C3A
:103BE000984211DA015D451CFA39012906D8AB4229
:103BF00006DD2118497801391F2901D92800EFE78E
:103C00000100251A461C02D10023136006E0665C01
:103C10006E5401318B42FADC181A106070BDC04638
:103C2000080D0020140D002010B5FEF7FBF9064B1F
:103C30001A68904201D200221A601B68C01A034B16
:103C400083428041404210BD100D0020204E0000F4
:103C500010B5094C094A2368126893420BD0084AF0
:103C6000D05CFEF725FB002805D0236801339B05B7
:103C70009B0D2360EDE710BD1C110020040D0020FA
:103C8000FA08002010B50400064B074A1B681268AA
:103C90009B1ADB439B059B0DA34202DAFFF7D8FF7B
:103CA000F2E710BD040D00201C110020F7B506003E
:103CB0000191151E2FD05768B800441C0630FFF73D
:103CC000E1FFFB20FFF77AFF1C20FFF777FFF0B240
:103CD000FFF774FFE0B22412FFF770FFE0B2FFF7C6
:103CE0006DFF6B461879FFF769FF0026BE4212DAB6
:103CF000B300EB189C680136E0B2FFF75FFF2012BB
:103D0000C0B2FFF75BFF2014C0B2FFF757FF200ED1
:103D1000FFF754FFEAE7F7BD70B5074D2C68092C93
:103D200008DC0C236343054E01349851F3185960A5
:103D30009A602C6070BDC04620110020142600201F
:103D4000F0B589B004900E0001284BDD284B0868BF
:103D50000293830709D1042807D90F23026813406F
:103D6000042B02D1FEF75AFB0290214B706803939B
:103D7000830709D1042807D90F2302681340042BB5
:103D800002D1FEF74BFB039000271A4B1A4D1B681C
:103D90000593059B9F4225DA2B1F0299186805F0B1
:103DA000BFFB00281BD12B686C6806930190019B18
:103DB000069A934213DA20680399079405F0B0FB42
:103DC0000834002807D131000498079B08315B684C
:103DD0000238984709E0019B01330193E7E7013777
:103DE0000C35D6E71B20FCF7AFFB09B0F0BDC04691
:103DF000A6AA0000201100201826002010B5FEF70A
:103E0000F3FFFEF715FAFEF7A7FBFEF7DDFBFFF762
:103E1000C9FE00F0C3FD00F081FF10BD962210B571
:103E200012010021034804F060FF0022024B1A60D7
:103E300010BDC0467C120020CC020020064B074A71
:103E40001B6812689B1ADB439B059B0D0122834272
:103E500000DC002210007047040D00201C1100201F
:103E6000F8B505000C0016001F1E0ED10320FFF749
:103E7000E5FF002827D0FA20FFF7A0FEE8B2FFF701
:103E80009DFEE0B2FFF79AFE1DE0501DFFF7D6FF42
:103E9000002818D0FB20FFF791FEE8B2FFF78EFE56
:103EA000E0B2FFF78BFEF0B2FFF788FE3012C0B22F
:103EB000FFF784FE3C00E31B9E4204DD2078FFF701
:103EC0007DFE0134F7E7F8BD70B50024F0250B4BFB
:103ED0001B689C420EDA2A006243094BD3181A78F9
:103EE000002A05D05978002311201A00FFF7B8FFE7
:103EF0000134ECE7FFF792FF70BDC046CC02002012
:103F00007C12002070B5060001250C4CB44212D082
:103F10002378002B0AD0002361781A001120FFF7C4
:103F20009FFFF0220021200004F0DFFE0135F03475
:103F30000B2DEBD170BD024B1D60F7E77C1200200A
:103F4000CC0200200123F3B50400FFB00D001000E7
:103F50001A420DD002AA1370431002A953704212E4
:103F60001B0E40148A700B71C8700B00052273E0A1
:103F7000032313401ED1042A1CD90F2201680A40D2
:103F8000042A17D1023302AA1370FEF747FA06007B
:103F900005F0D8FAF823FF33984200DD180000231B
:103FA000834205DA01335A1EB25C02A9CA54F7E70C
:103FB000421C50E0042801D0002809D1032302AAA2
:103FC000043813704342434153701300022243E00C
:103FD000002B45D1042843D90F210268114005293F
:103FE00012D1043302A90B70F8231209FF33920097
:103FF0009A4200DD1A00002393422BDA0133C118E4
:10400000C97802AEF154F7E7062929D101390E002B
:10401000120956430196F826019FFF36B7421FDC6E
:1040200002AE31700136934213DA01270133990051
:104030004158394201D0394100E00A49012737701F
:104040000F127170B7700F14090EF77031710536C9
:10405000E9E7019A013202AB29002000FFF700FFD7
:104060007FB0F3BD19FCFFFF70B5F02305000024FD
:104070000D4A1800604380184178A94203D00134EA
:104080000A2CF6D10FE0F022002104F02EFE074AA0
:104090001368013BA34200D11460002329001A00D9
:1040A0001120FFF7DDFE70BD7C120020CC02002045
:1040B00010B5B2B002236A460400137005F042FA4C
:1040C000C72800DDC7200023834205DA6946013393
:1040D0005A1EA25CCA54F7E7421C6B46FE2114200C
:1040E000FFF7BEFE32B010BD30B5B3B002236A4652
:1040F0000500137005F026FA041EC72C00DDC72446
:104100000023A34205DA694601335A1EAA5CCA5449
:10411000F7E720003230FFF7B5FD621C6B46FF2148
:104120001420FFF79DFE33B030BD0000F7B5234BE0
:1041300006001B68F020009300232149009A934257
:104140000ADA02005A438A185478B44202D112782B
:10415000002A31D10133F1E70024F0231A00624331
:1041600001920199164A55182F78002F06D0013474
:104170000A2CF3D11348FFF7B7FF1DE0F0223900F6
:10418000280004F0B2FD02230D4A0199EB6053545C
:104190000D4AF1008A58009B6E70AE70AA602F61C4
:1041A0006F61A34202DC054B01341C600023310027
:1041B0001A001020FFF754FEF7BDC046CC020020C5
:1041C0007C1200201BAC0000DC1B002010B5FFF7A8
:1041D0007BFE0024064BE200D3181B79043B012B25
:1041E00002D8E0B2FFF7A2FF0134FF2CF2D110BDDC
:1041F000DC1B0020F7B50E0000247F250190194B31
:10420000E200D1180979062901D0032926D198584E
:1042100083682B401C2B21D1C3681A002A40042A32
:104220001CD102692A40192A18D11B0A01339B00AC
:104230000C30C018FEF7F2F8070005F083F90023F0
:10424000B0420BD19E4206DD019AF95CD25C9142EC
:1042500004D10133F6E7E0B2FFF768FF0134FF2C29
:10426000CDD1F7BDDC1B002070B505000024064B46
:10427000E200D3181B79AB4202D1E0B2FFF756FF40
:104280000134FF2CF3D170BDDC1B0020F7B5FDF726
:10429000C9FE514B1A68904201D200221A601A6876
:1042A0004E49821A8A4200D894E01860FDF7C4FE95
:1042B000071E00D101370020FDF790FF019000207C
:1042C000FDF7A0FF019B0090454C464D002B17D0F9
:1042D0002368002B7AD12B682760002B72D0424BC9
:1042E00001261B78002B06D10920FFF7BDFF3F4BAD
:1042F0001E703D4B03E00720FFF7B6FF3B4B1E70DF
:10430000009B002B16D02B68002B13D123682F6045
:10431000002B22D0354B01261B78002B05D109201C
:10432000FFF7A2FF314B1E7002E00820FFF79CFF51
:104330002D4B1E702368002B0FD02C4E3278002A94
:104340000BD19F4200D227602368FB1A312B04D97E
:104350000720FFF789FF012333702B68002B0FD054
:10436000214E3278002A0BD19F4200D22F602B6859
:10437000FB1A312B04D90820FFF776FF0123337095
:104380002368002B0CD0019B002B09D1174E3378EA
:10439000002B02D10720FFF767FF00232360337053
:1043A0002B68002B16D0009B002B13D10E4B1A78D4
:1043B0001C00002A02D10820FFF756FF00232B60C3
:1043C000237007E0009B002BA0D1B3E7009A002ADE
:1043D00099D1B2E7F7BDC046FC0C00200F270000C2
:1043E000000D0020141100200C0D002018110020D9
:1043F00037B500240500FFF767FD01A80194FDF71C
:10440000DBFE21002000FEF7D5F9FEF793FBFDF758
:104410000DFFFDF70CFFFEF7E1FCFDF731FEA542B5
:1044200004D0FDF75BFF0248FFF75EFE37BDC046D4
:1044300030AC0000002310B501001A001120FFF776
:104440000FFD10BD07B56B46197069465A701312FF
:104450008B701314120ECB700A716B46010005228B
:104460001320FFF7FDFC07BD10B50A000100122064
:10447000FFF768FD10BD70B5050008000C00323074
:10448000FFF700FC2B00220000211B20FFF7E8FCB7
:1044900070BD10B50C000300110014202200FFF7BE
:1044A000DFFC10BD70B506000020FEF739FD0024CA
:1044B000FF25002810D003681A142A40152A05D1B8
:1044C0001B122B40B34204D1040002E01D2A00D18C
:1044D0000024FEF725FDECE7200070BDF0B5802735
:1044E0009DB0FFF7B5FBB64DB64C2868FF00391AF2
:1044F0002018FDF7C3FE2B680600C3182B60002BA5
:1045000000D1D9E1002E0DDD2868391A2018FDF7F9
:10451000B5FE2B6806001B182B60FDF783FDAA4B28
:104520001860EFE72378FA2B00D00CE12B68022B00
:1045300006DCFFF779FB002800D1BDE10120B6E1E0
:104540006078A5780238182800D9FAE002F0FEFC5D
:104550000D1E22262932F93D67F96F83D4E5F9F95A
:10456000F9F9F9F9F9F9F9F9F300FF2D00D1E8E0CB
:104570002800FFF779FD00229449EB005A50CB1830
:104580001A7129000092130013204DE02800FFF754
:10459000CDFDD6E02800FFF767FDD2E0FFF716FE5D
:1045A000CFE0FFF791FC0020FFF722FF8848FFF7DC
:1045B0009BFDC6E0632D00D9C3E0864BAA00D2580C
:1045C00029001520FFF7BEFCBBE000242000FFF708
:1045D00069FF071E03D10134642CF7D1B1E0083024
:1045E00004F0B0FF06000530FFF74CFBFB20FFF79F
:1045F000E5FA1D20FFF7E2FAE0B2FFF7DFFAF0B2CA
:10460000FFF7DCFA3012C0B2FFF7D8FA0025AE424D
:10461000E1DD7B19187AFFF7D1FA0135F7E70021C0
:104620001D200B000A000091FEF786FE89E0FDF7D1
:1046300013FD03AC684A64210090684B200004F02D
:104640001BFF02232000237004F07CFF23000200E4
:104650000021162073E000245C4AE300D558002DA9
:1046600046D06B689E00701DFFF70CFB2B000025E9
:104670003200083321000120FFF7F2FB0020FEF793
:104680004FFC2E002F0000281DD0FF2103681A12B6
:104690000A40A24214D11A140A400B2A07D10B4037
:1046A0000DD0012B09D0022B00D103E108E0132A21
:1046B00006D100252E002F0002E0060000E00700D2
:1046C000FEF72EFCDFE7002E04D03200012120008F
:1046D000FFF7ECFA002D04D02A0002212000FFF79A
:1046E000E5FA002F04D03A0000212000FFF7DEFA9F
:1046F0000134FF2CB0D124E00024FFF7E5FB2200B9
:10470000210000942300DA20FEF716FEFF2221008C
:10471000D2002E4804F0E9FA13E0012D02D1FEF791
:1047200025FD0EE0022D02D1FEF76AFE09E0012010
:10473000FFF75EFE05E0002329001A001A20FFF7AC
:104740008FFB0320B3E0FB2B00D0F7E62A68042A96
:1047500000DCEEE62679E078214B360206439E42E5
:1047600000DDEBE6331D9A4200DCE2E6E35CFE2B63
:1047700000D0E3E66378A578711E1B2B5DD004D8CA
:10478000012B08D0082B2DD090E01D2B64D058D3DE
:104790001E2B7BD08AE0FF2D00D187E02800FFF799
:1047A00063FC67790634B31E290000943A000A209E
:1047B000FEF7C2FD054BED00E8505D192F7175E065
:1047C000080D0020140D0020100D0020DC1B00201F
:1047D0003FAC0000D423002056AC000051AC0000D8
:1047E000F6030000632D61D86079022813D00328F6
:1047F0001BD001285AD1A71D7A78A479BB78120260
:1048000022431B0413431A00FB78AD001B0613431D
:104810005B0003430EE0002948DDB11EA01DFDF73B
:10482000E1FD264BAD00E85040E0A379AD005A1EF3
:1048300093419B00214AAB5038E0601DFFF7DAFC42
:1048400034E06279FF2D31D0022A2FD80634B31E0E
:10485000009429000B2016E00B1E632B00DD632360
:10486000002203A8934204DDA11849798154013242
:10487000F7E7D9430022C917194041180A70009080
:10488000290015200133FEF757FD0FE0012D0DD152
:1048900000290BDD6379002B03D0322B02DD32239C
:1048A00000E02B0064225343054A1360701DFFF79C
:1048B00093F901E0050003E71DB0F0BDD42300200B
:1048C000040000200122094B1A60094A1368002BDA
:1048D000FCD00322074B1B68D8171040C0180123D7
:1048E00080100638400018437047C04600C00040A2
:1048F00000C1004008C500400120704710B5064CBB
:10490000200000F041FB0549200000F061FB01227E
:10491000034B1A6010BDC0464C110020801A0600DF
:104920002411002010B501210D20FDF79BFB012172
:104930000E20FDF797FB00210F20FDF793FB044CA1
:10494000200000F05DFA1021200000F075FA10BD83
:104950003811002010B504680D20E30703D564105A
:10496000FF2C03D91720FBF7EFFD06E0FFF7DAFF76
:10497000E1B2024800F082FA002010BD3811002098
:1049800010B5FFF7CFFF0021034800F077FA0123AD
:104990004000184310BDC0463811002010B5034A2E
:1049A00007210348FFF7B8F910BDC04648010020B1
:1049B0005DAC00000D4B70B51B6804000E001500C7
:1049C000002B01D1FFF79AFFE1B2094C200000F063
:1049D00087FBF1B2200000F098FAE9B2200000F065
:1049E00094FA200000F0E6FB70BDC04624110020C0
:1049F0004C11002010B501240368234205D0416802
:104A0000214202D08268224201D10D2004E05810D8
:104A10004910802803D91520FBF796FD0BE0FF29EC
:104A200001D91620F8E75210FF2A01D91720F3E721
:104A3000FFF7C0FF002010BDF7B501242300A042FE
:104A400037DD0A68144234D01B4B55101B684C6884
:104A5000002B01D1FFF752FF0127184EE9B23000B9
:104A600000F03EFB3C4205D03C413000E1B200F09A
:104A70004CFA1AE00325254017D1042C15D90F2331
:104A800022681340062B10D113090193019B9D420C
:104A90000BDAAB00E3185968394204D04910C9B2A7
:104AA000300000F032FA0135F0E7300000F082FB10
:104AB00000231800FEBDC046241100204C11002028
:104AC000144B70B51B6805000E00002B01D1FFF7D9
:104AD00015FF114CEDB22900200000F001FBF1B2EE
:104AE000200000F012FA0021200000F005FB002851
:104AF00001D040420CE001222900200000F0EBFA36
:104B0000200000F0F8F90028FAD0200000F0F8F9B1
:104B100070BDC046241100204C11002010B50124A6
:104B20000368234202D04168214201D10D2004E0F4
:104B300058104910802803D91520FBF705FD07E020
:104B4000FF2901D91620F8E7FFF7BAFF40002043FC
:104B500010BD0000002370B5344D0400EB56013346
:104B60002BD10D211D20FFF7ABFF5A2804D10122C4
:104B70002A212A703D380AE00F211920FFF7A0FFF3
:104B8000332807D102235F2220212B701A38FFF728
:104B900011FF12E00D211E20FFF792FFC7280AD156
:104BA000032300222A21A9382B70FFF703FF1B22C1
:104BB0002A211E20EBE700232B700023EB56022B4B
:104BC00006D0032B13D0012B26D121001D2010E08D
:104BD000012C04D129211920FFF772FF0DE0032CCD
:104BE00015D12B211920FFF76BFF043C05E02100B4
:104BF0001E200124FFF764FF64427F2801DD013895
:104C0000FF3803007F330ADA7F20404207E0052C9B
:104C100002D12D211920ECE70124002064426423F5
:104C20007F21584302F026FA604370BD4401002002
:104C300010B50120FFF78EFF01234000184310BD7F
:104C400010B50320FFF786FF01234000184310BD75
:104C500010B50520FFF77EFF01234000184310BD6B
:104C6000F8B501263400B04236DD0F683E4233D03D
:104C70004D68AB0730D1042D2ED90F232A6813407D
:104C8000062B29D1154B1B68002B01D1FFF736FEEF
:104C90000024354204D12B681C09202C00D9202483
:104CA0000F4E7F10F9B22200300000F014FAA70076
:104CB000EF19AF420DD0300000F01DF90028FAD0F6
:104CC000300000F01DF901234000184368600435EE
:104CD000EFE70120640004432000F8BD2411002008
:104CE0004C110020002070470020704700207047C2
:104CF0000020704700207047002070470020704758
:104D00000020704700207047002070470020704747
:104D100000207047704770477047000010B5034A85
:104D20000C210348FEF7F8FF10BDC04680010020AB
:104D30009EAC000010B5FDF787FA0648FDF7F2FAC1
:104D4000FFF75CF80448FFF7CFF9FEF75DFBFFF7CC
:104D50003DFA10BDE204000014AD000010B5FDF7EF
:104D6000FBF810BD70B5002504AC24780573A9428A
:104D700005D10A4B0A4A23210A4803F02DFF01609E
:104D80000949920052589B0002715B588371A3003D
:104D90005B58856043710223C37170BD69AD00002B
:104DA0002CAD000077AD000000AE0000037B002BAF
:104DB00004D14373837303610133037370470000AD
:104DC0001FB50191A02100240068C900D2B244504F
:104DD000012A07D0A24203D0032A05D1042202E00F
:104DE000022200E006221343034A8350034B019A38
:104DF000C250012343501FBD54050000240500008C
:104E000010B50400FFF7D2FFA1222368A179D200D8
:104E100099506179064A20009950217904329950BD
:104E2000044B19685A689B68FFF7CAFF10BDC0465B
:104E30000C0500002C1100204BB2002B0CDB802352
:104E40003F290CD81F290CD80F290CD807290CD8BA
:104E500003290CD81B060BE080239B0408E0DB042D
:104E600006E01B0504E05B0502E09B0500E0DB05B6
:104E70000168014A8B507047240500000368074A07
:104E800099501A00FC32D1680029FCD0A321C90036
:104E900058580023C0B2D3607047C0461C050000BC
:104EA00007B58022074BD2051A6000229A600232B1
:104EB0001A710F230C3200930349023B0348FFF79A
:104EC00051FF07BD2C110020003000403811002098
:104ED000F8B505000E0017000024BC4208D02B686E
:104EE000315D1B6828009847002801D00134F4E7A1
:104EF0002000F8BD704710B51C3001F0CDFB10BD8F
:104F000010B51C3001F0BAFB10BD70B5437E0D002A
:104F1000002B05D06430040001F0CDFB002801D047
:104F2000002004E02000290001F099FB012070BD61
:104F300010B51C3001F0B6FB10BD0000F7B50193B1
:104F4000FA23002504009B0083600D4B4560083365
:104F500003601C300F00160001F076FB2000643067
:104F600001F072FB074AB600B35827616375019BD5
:104F700020009B009B586576A576A375FEBDC046B4
:104F8000E0AD000000AE00000123A022C375837DC8
:104F90000C49C133FF33D2059B009950437DC13387
:104FA000FF339B009950CC210369074A490499506B
:104FB0000521243A9950817D08329950417D034A58
:104FC000995070470C060000240500000C050000F5
:104FD000A02302690020DB00D0500948814204D997
:104FE0000848814204D9CD2103E0CC21490401E0E5
:104FF0008021C904044811500521D1507047C04692
:10500000A086010090D0030024050000F7B505003C
:1050100000200C00019382425CD0161E402E00D965
:1050200040262F001C37380001F024FBB1222B69E9
:10503000D20080219C50012289005A50A97E00296B
:1050400001D11A621A600024731E2A69A34206D194
:10505000019B002B03D0802302219B00D150012310
:1050600013621300FC33D968002902D1996A002920
:10507000F9D0996A00290AD1D960A323DB00D1585D
:105080003800C9B2013401F0EAFAA642DCD8019A2C
:105090002B69002A04D11A00FC32916A00290AD037
:1050A00001210022AA7659611900FC318868002884
:1050B000FCD08A6007E00121A976D961D16C002972
:1050C000FCD00021D164FC339A6A002A01D000226E
:1050D0009A62E0B2FEBD10B50123FFF797FF10BD45
:1050E0000300AC3310B504001970643001F0C2FA4B
:1050F0000123637610BD0000F8B500220D00010009
:105100004276AC31036904000878B121C9005850D7
:10511000802189005A5001321A629A602600643652
:10512000300001F0B9FA00280ED03000276901F0F4
:10513000A5FA1E4BF8502369FC331A6A002A0CD1D9
:105140009A6A002AF9D008E02369002D0AD11A00D2
:10515000FC32916A002905D10EE09A6A002AF3D147
:105160001A62DBE701225A611A00FC3291680029B9
:10517000FCD00021916006E00121D961D16C0029A9
:10518000FCD00021D1641A000020FC32916A8142D7
:105190000BD0074990625A5802305A50824204D0CC
:1051A000043A534253410230C01AF8BD1C050000B6
:1051B000C404000010B50121FFF79EFF10BD0000E0
:1051C00010B51323142202490248FFF7B7FE10BDA1
:1051D000004000404C110020F0B5474680B4CB0F92
:1051E00098464A4C4B005B0D1E1982B007000A001E
:1051F000132E35DC002E57DB454B040033411F00D6
:105200000F4007430D00002F24D05B081C000C400A
:1052100020430027002807D0132E00D172E08022FF
:10522000D202324199430A434346DE00394B110012
:105230009E1934687568380022002B0002F0DAF9F4
:10524000009001910098019922002B0003F086F84C
:1052500004000D002000290002B004BC9046F0BDFF
:10526000332E0CDD802304000D00DB009E42F1D1C3
:1052700002000B0002F0BEF904000D00EAE7264C24
:105280000D00A446012463446442DC40A446614608
:1052900004000142DED049080142C5D08027FF0545
:1052A0001F4188430743BFE74B005B0803430400EB
:1052B0000D00002BCED00B031B0B03435A421343AC
:1052C00080221B0B120313404A0C52041343190093
:1052D0004346104ADB00D3181C685D6822002B008F
:1052E00002F088F9009001910098019922002B00AA
:1052F00003F034F842464B005B08D6073343040002
:105300001D00A7E780273F0689E7C04601FCFFFF95
:10531000FFFF0F0088AE0000EDFBFFFF30B5214A14
:105320004B0087B05B0893421EDD1F4A934205DDA8
:1053300002000B0003F012F807B030BD02AA00F023
:1053400035F803231840049A059B01281ED0022833
:1053500011D000281FD00298039900F02DFA802365
:105360001B069C466144E7E70023002200930023CC
:1053700000F088FFE0E7012402980399009400F010
:1053800081FF80231B069C466144D5E70298039960
:1053900000F012FAD0E7012402980399009400F07B
:1053A00071FFC9E7FB21E93FFFFFEF7FF0B54E46F4
:1053B00057464546E0B4DC4B4E0090B01700894696
:1053C00076089E4200DC81E0D84B9E4220DCD84A21
:1053D000002900DC89E1D74B02F0C0FFD54B040067
:1053E0000D009E4200D18AE0D34AD44B02F0B6FFB2
:1053F00002000B0020003A607B60290002F0AEFF43
:10540000CD4ACE4B02F0AAFFB860F960012066E0F9
:10541000CB4B9E4200DC8DE0CA4B9E4265DCCA4904
:1054200032158A46924453461B05F51A290004009A
:1054300003F0E8FA03F01CFB02000B002000290037
:105440000A920B9302F08AFF0022C04B02F00CFD7F
:105450000290039103F0D6FA03F00AFB04000D005A
:1054600002000B00029803990C940D9502F076FF50
:105470000022B64B02F0F8FC002200230E900F91A0
:1054800001F002FF002800D14CE10023002220009F
:10549000290001F0F9FE0222431E9841131AAC4A7A
:1054A0003900019202220AA80092524600F09EFAA8
:1054B0004B46002B13DA8022120694467B6840424A
:1054C00063447B60FB686344FB6008E002000B0000
:1054D0003A607B60002200230020BA60FB6010B0BD
:1054E0001CBC90469946A246F0BD02000B0002F09B
:1054F00035FFB860F960386079600020EFE7D322AB
:105500008E4B520502F02AFF924A934B04000D0085
:1055100002F024FF02000B0020003A607B602900AB
:1055200002F01CFF8B4A8C4B02F018FFB860F96048
:105530000120D4E700F056FF884A894B04000D0093
:1055400002F092FC0022874B02F054F803F05AFA62
:10555000804603F08DFA764A764B0690079102F06A
:1055600083FC02000B002000290002F0F7FE734BC1
:1055700002900391069807996F4A02F075FC434622
:1055800004000D00049405951F2B30DC013B764A86
:105590009B009B589E422AD002000B000298039960
:1055A00002F0DCFE02000B0005000C003A607B609C
:1055B000029803992A00230002F0D0FE049A059B6A
:1055C00002F0CCFE06000B003200BA60FB604B46D6
:1055D0004046002B00DB82E780231B069C46644488
:1055E00061443D607C60BE60F960404277E7049AA8
:1055F000059B0298039902F0B1FE0B0002003A608D
:105600007B604B0036155B0D05000C00F31A102B68
:10561000CEDD06980799D322484B520502F024FCB0
:1056200004000D0002000B000298039902F096FEA0
:1056300002000B00029803990892099302F08EFE73
:1056400022002B0002F08AFE04000D000698079944
:10565000404A414B02F008FC22002B0002F07EFE83
:1056600002000B00049005910898099902F076FE5B
:1056700002000B003A607B604B005B0DF61A0500E0
:10568000089A099B0C0002920393312E90DD069834
:105690000799B822304B920502F0E6FB04000D009A
:1056A00002000B000298039902F058FE0A00010064
:1056B00013000291039202000898099902F04EFE2D
:1056C00022002B0002F04AFE04000D000698079904
:1056D000264A274B02F0C8FB22002B0002F03EFEB8
:1056E00002000B000492059358E7124B01F082FF71
:1056F000104B04000D009E423CD00F4A0F4B01F0AE
:1057000079FF02000B0020003A607B60290002F064
:1057100025FE094A094B01F06DFFB860F9600120D0
:105720004042DCE60323BAE6FB21E93F7BD9024095
:1057300000004054FB21F93F3163621A61B4D03D4F
:10574000FB213941FFFFEF7FEAFBFFFF00007041C3
:1057500018AF00007370032E8A19A33B83C8C96D6C
:10576000305FE43F0000E03F98AE0000C1492025D3
:105770009A837B39D3220D4B520501F03BFF0C4A33
:105780000C4B04000D0001F035FF02000B0020005F
:105790003A607B60290002F0E1FD054A054B01F00B
:1057A00029FFB860F9600120404298E661B4D03D1D
:1057B0007370032E8A19A33BF0B54F464646C0B41A
:1057C00087B000920193754B4F00814688467F0851
:1057D0009F4263DC03F016F9002800D1DAE04A4664
:1057E00043464846414602F03FFB04000D006C4A28
:1057F0006C4B02F039FB6C4A6C4B01F0FBFE220053
:105800002B0002F031FB6A4A6A4B02F0A7FD22002E
:105810002B0002F029FB684A684B01F0EBFE2200E6
:105820002B0002F021FB664A664B02F097FD220036
:105830002B0002F019FB644A644B01F0DBFE2200EE
:105840002B0002F011FB029003910022604B20001C
:10585000290002F009FB029A039B06000F002000BA
:10586000290002F001FB009A019B04000D0048464C
:10587000414602F0F9FA02000B002000290002F074
:105880006DFD02000B003000390002F067FD0200E0
:105890000B0000204F4902F061FD70E002000B0098
:1058A00002F0E2FA04000D003D4A3E4B02F0DCFA41
:1058B0003D4A3E4B01F09EFE22002B0002F0D4FA3E
:1058C0003B4A3C4B02F04AFD22002B0002F0CCFA8E
:1058D000394A3A4B01F08EFE22002B0002F0C4FA46
:1058E000374A384B02F03AFD22002B0002F0BCFA96
:1058F000354A364B01F07EFE2B00220002F0B4FA4E
:10590000354B029003919F429FDD344B00229F4212
:105910003ADC334900207B182E4916001F0002F0A4
:105920001DFD049005910022294B2000290002F062
:105930009BFA32003B0002F011FD029A039B060025
:105940000F002000290002F08FFA009A019B04004A
:105950000D004846414602F087FA02000B00200085
:10596000290002F0FBFC02000B003000390002F0BD
:10597000F5FC02000B000498059902F0EFFC07B05B
:105980000CBC90469946F0BD164B00260492059338
:10599000154FC8E700200F49F1E7C046FFFF3F3E23
:1059A000D43888BEE9FAA8BDC4B1B4BD9EEE213E8C
:1059B000AD529C804F7E923E9015CB19A001FA3ECD
:1059C0007751C1166CC1563F4C5555555555A53F9D
:1059D0000000E03F0000F03F3233D33F0000E93FDA
:1059E0000000E0FF0000E73F0000D23FF0B5564660
:1059F0004D4644465F46F0B48E4CA54409911900CB
:105A00001400A89A0B938C4B9200D2580B00029072
:105A1000013BE01E18211D0016000892009301F0C2
:105A200029FBC3430200DB171A40130011000133A6
:105A30000E929A009B1ADB001B1906934C1B7619D9
:105A400018D4A99BA5009C46361926AF654401369B
:105A500007E0286803F00CF8013403C70435B442AA
:105A600008D0002CF5DA00200021013403C70435EA
:105A7000B442F6D1089B002B01DA00F0F9FB76ABBB
:105A800019008B4626AA9146089A0A930132D20041
:105A90009344029A9A469046009BDB00994408334F
:105AA0009844009B002B00DAB5E14C460026002705
:105AB000029D2268636803CD02F0D6F902000B0054
:105AC0003000390001F096FD083C06000F00454506
:105AD000EFD15346C0C39A4608239C46E144DA45B9
:105AE000DFD10899554A0B00944663449B0012A8E5
:105AF00084461A000298624483460D920B9A04333E
:105B0000D200634493440F930591059A0A98D300F9
:105B100019000C938C46030063441E685F68002ADA
:105B200034DD12AB99461300454A804694466344DF
:105B3000DB00984474AB9A460022424B3000390097
:105B400002F092F902F05EFF02F092FF00223E4B5B
:105B500004000D0002F088F902000B00300039004B
:105B600002F0FCFB02F04EFF4B4601C39946434650
:105B700020001A685B68290001F03CFD08235B42A5
:105B80009C46E04406000F00D045D5D1069B30006E
:105B90001A003900994600F0C1FCFF2300229B0542
:105BA00004000D0002F060F900F020FC0022274BF9
:105BB00002F05AF902000B002000290002F0CEFB8F
:105BC00004000D0002F01EFF804602F051FF0200AB
:105BD0000B002000290002F0C1FB4C4606000F001C
:105BE000002C00DCF8E0059B18205A1E920012AB36
:105BF0009B58001B19000141884481405B1A12A97F
:105C00008B501722121B13410793079B002B4BDD70
:105C100001239C46059BE044002B00DCF2E280253A
:105C20001096119712AB0021002409486D04059FBE
:105C300019E0C04684FDFFFF20B00000FEFFFF3FDB
:105C4000FFFFFF1F0000703E000070410000204079
:105C5000FFFFFF00002A02D0AA1A1A6001340131A6
:105C600004338F4209DD1A68002CF3D0821A013107
:105C70001A60012404338F42F5DC109E119F069BAD
:105C8000002B0EDD012B00D1B1E0022B09D1059BC9
:105C900012A95A1E920012AB9B5810939B029B0AAA
:105CA0008B50079B022B7ED000230022300039004E
:105CB00001F0EAFA059B002800D16BE208995A1E10
:105CC000914210DCBF490F988C4612A963448C4660
:105CD00000219B0063441C68043B21438342FAD1AA
:105CE000002900D0B5E0089B12AA013B9B00D358C5
:105CF000002B00D084E201220D9B043B5968013245
:105D00000029FAD005990B008C46013362440792B2
:105D1000934242DC0E9A9446A99A634492460B9AA7
:105D20009B00944626AA90469A44059B0A9A63448F
:105D3000DB0098440C9B94469946079BE144DB00AA
:105D4000634405935346186802F092FE4346186078
:105D50005960009B002B23DB444600260027029D50
:105D60002268636803CD02F07FF802000B00300068
:105D7000390001F03FFC083C06000F005D45EFD103
:105D80004B469E60DF6004239C460433E2449C46FD
:105D9000059BE144E0449945D4D1079B0593B4E6C3
:105DA00000260027ECE732003B000020864902F085
:105DB000D5FA06000F00002C00D175E7069A0020E6
:105DC000814900F0ABFB02000B003000390002F00B
:105DD000C5FA06000F0067E7069B002B12D1059B52
:105DE00012AA013B9B00D558EB1507930DE7059BC5
:105DF00012A95A1E920012AB9B5810935B025B0AC9
:105E00008B504EE70022714B01F062FA00280ED150
:105E10000023079348E7534600260027C0C39A464D
:105E200008239C46E144DA4500D03AE659E60123CE
:105E30009C4601330793059BE044002B00DDEEE612
:105E400032003B000020604902F088FA06000F0093
:105E50002AE743460B93069B12A8183B19000693AA
:105E60009300C3580092002B0FD15648130084466C
:105E700012A8634484469B006344043B5868013A7B
:105E800018390028F9D000920691069A00204E4950
:105E900000F044FB009B04000D00002B00DAB3E18E
:105EA00012AA94469F00DB0067449C460A9A059319
:105EB000624493461600386802F0DAFD22002B0097
:105EC00001F0D2FF424B30607160002220002900B7
:105ED00001F0CAFF083E74AB04000D00043FB3425A
:105EE000E9D100239A464EAB0293089B99464B4654
:105EF00000260027002B21DB8020364B5D4698468C
:105F0000C005354900260027002408E008239C46E8
:105F10000835E044A24511DB4346186859682A68F1
:105F20006B6801F0A1FF02000B003000390001F0A6
:105F300061FB013406000F00A145E7DA029A5346DF
:105F40009446DB0063441E605F6001239C46093B6E
:105F5000E2449C4674ABE3449B45C8D1029B9946FE
:105F6000A89B022B00DD82E0002B37DC1DD1059BB6
:105F700000254B441E00002432687368280021006D
:105F800001F038FB009B05000C00083E5A1E0092F1
:105F9000F2D2079B002B03D080231B069C4664444F
:105FA0002A00230009990A604B6007200B9B1840C8
:105FB0009F239B009D443CBC90469946A246AB461D
:105FC000F0BDC046FFFFFF3F0000F03F0000E03F94
:105FD0000000703E30B00000FB21F93F059B00201F
:105FE0004B441E0000214CAF32687368083E01F03C
:105FF00001FBBE42F8D1079B002B24D08023099AD5
:106000001B06CB18106053600B0002004E984F998E
:1060100002F0A4F9009B002B0BDD012450AD0CCD48
:1060200001F0E8FA009B0134A342F8DA079B002B49
:1060300003D080231B069C4661440B000200099993
:106040008A60CB60B1E702000B00099C22606360AC
:106050000B0002004E984F9902F080F9009B002B34
:10606000DBDC0B00020009998A60CB609DE7A89BEE
:10607000032B9AD1009B002B00DCE3E07E4A059BBA
:1060800094464B441E685F68009B63449A46DB005D
:106090004B4498464CAB9B4643465C681B681800D3
:1060A000210032003B000290039101F0A3FA0400AA
:1060B0000D0002000B000298039902F04FF93B001B
:1060C000320001F097FA43469860D9601C605D6029
:1060D00008235B429C46E04426002F00C345DBD1E9
:1060E000009B012B00DCADE0059BC8464B441E68BD
:1060F0005F685346DB009B46D844434630005C68EB
:106100001B683900009301941A00230001F072FA11
:1061100004000D0002000B000098019902F01EF926
:106120003B00320001F066FA43469860D9601C607B
:106130005D6008235B429C46E04426002F00C14579
:10614000DBD15D460027002408354D4450AE2A6857
:106150006B683800210001F04DFA083D07000C0083
:10616000AE42F4D1079B002B71D0099A4E994B4651
:106170001160802109068C465B6849466344536080
:106180004B46DB688968634464449160D36017615F
:1061900054610AE7994643460B93069B30005A42E6
:1061A000390000F0BBF90022344B04000D0001F06F
:1061B0008FF8002832D0324B00222000290001F055
:1061C00053FE02F01FFC4A460600970002F050FC06
:1061D00000222A4B01F048FE02000B00200029009B
:1061E00002F0BCF802F00EFC12AAD0514A46069BFF
:1061F0000132183300920693930012AAD65044E657
:1062000001227FE500243AE5A89B022B14DC002B39
:106210000FDC00D0C9E600250024BAE64B4620007A
:1062200029009E0002F0EEFB12AB98514B46009302
:106230002BE600200021DEE64EAB9946A89B032BFF
:1062400000D0B2E6079B00270024002B8DD14E9A88
:106250004F9B09990A604B604B469A68DB68009235
:1062600001938A60CB603A0023000A614B619CE68F
:1062700076AB0A9335E4C046FFFFFF1F0000704174
:106280000000703EF0B54F464646C0B487B000925D
:106290000193464A4B00814688465B08934205DCE1
:1062A00002F0B0FB4146031E484666D04A464346CC
:1062B0004846414601F0D8FD04000D0002000B00E5
:1062C0004846414601F0D0FD394A3A4B06000F00DE
:1062D0002000290001F0C8FD374A384B02F03EF893
:1062E00022002B0001F0C0FD354A364B01F082F947
:1062F00022002B0001F0B8FD334A344B02F02EF897
:1063000022002B0001F0B0FD314B324A01F072F94E
:106310000E9B02900391002B34D00098019900222B
:106320002D4B01F0A1FD029A039B049005913000D2
:10633000390001F099FD02000B000498059902F064
:106340000DF822002B0001F08FFD009A019B02F056
:1063500005F8224A04000D00214B3000390001F0FD
:1063600083FD02000B002000290001F043F9020028
:106370000B004846414601F0F1FF07B00CBC9046C7
:106380009946F0BD02000B002000290001F06CFDD1
:10639000124A134B01F0E2FF32003B0001F064FDB2
:1063A0004A46434601F026F9E7E7C046FFFF3F3E75
:1063B0007CD5CF5A3AD9E53DEB9C2B8AE6E55A3E8F
:1063C0007DFEB157E31DC73ED561C119A0012A3F2B
:1063D0001111813FA6F810110000E03F49555555B5
:1063E0005555C53F49004B0819007047454AF8B557
:1063F000564692464B005B0D9A444D465F464446D6
:106400005246F0B4894605000C000E000700132A1E
:1064100022DC002A47DB52463B4B134198460B00D7
:1064200042461340034311D0384A394B01F0E2F899
:106430000022002300F042FF002805D0002C41DBA1
:106440004E46434600279E43380031003CBC9046F0
:106450009946A246AB46F8BD5246332A08DD802352
:10646000DB009A45F2D102000B0001F0C3F8EDE722
:10647000284A9446012263445242DA40934602423B
:10648000E4D0224A224B01F0B5F80022002300F0AC
:1064900015FF0028D8D0002C1ADB5B464E469F43E0
:1064A00038003100D2E7194A194B01F0A3F8002255
:1064B000002300F003FF0028C6D0002C16DB0027C5
:1064C0000026C1E7802352465B0313419944B7E796
:1064D0005346142B12D03423524601279B1A9F4057
:1064E0007F19AF429B415B429944D6E76400640840
:1064F00025430027002DA7D0074EA5E7133B9C4658
:10650000E144CAE701FCFFFFFFFF0F009C75008814
:106510003CE4377EEDFBFFFF0000F0BF4B0070B5A1
:106520005B0D14000A00002B1AD14B005B080343DB
:1065300015D00022224B01F097FC224B0A009C420E
:1065400022DB4B005B0D363B1F4DE318AB4220DCDA
:10655000002B0DDD1D4C1B0522401A43110070BDA0
:106560001B4DAB42F0D102000B0001F043F8F6E7FF
:106570001D00353518DA174B02009C420ADC0B006F
:106580001548164900F032F8134A144B01F06CFC20
:10659000E5E702000B001248124900F027F8104A04
:1065A000104B01F061FCDAE7084C363322401B0542
:1065B0001343190000220C4B01F056FCCFE7C046F4
:1065C00000005043B03CFFFFFE070000FFFF0F80BC
:1065D000FF07000050C3000059F3F8C21F6EA50169
:1065E0009C7500883CE4377E0000903C30B54A0042
:1065F000DB0FDB0752081A43110030BDF7B5060068
:106600000D000C008B180193019B671B9C4207D067
:10661000336821781B683000984701340028F3D193
:106620003800FEBD70B505000C00081E07D002F052
:1066300089FF2B6802005B6821002800984770BD25
:1066400010B5FFF7EFFF10BD10B540220021040088
:1066500002F04BFB002320002364636410BD3F2342
:10666000026C10B5541C2340446C9C4201D08154F0
:10667000036410BD0023036443647047436C026CE1
:10668000934206D03F21C25C01330B4043641000AB
:1066900001E0012040427047036C406C181A00D59D
:1066A00040307047436C026C934201D0C05C01E003
:1066B000012040427047036C406C5A1C3F2313403A
:1066C000181A42424241D0B27047000003210A48E2
:1066D00002680A430260094802680A4302600849E6
:1066E000084A094B9B1A03DD043BC858D050FBDC19
:1066F00000F012F8F9F73EFD240500405405004073
:1067000004B3000000000020AC020020FEE7FEE71A
:10671000FEE7FEE7FEE7FEE72D4B10B51A78012AEB
:1067200019D12C4A1268120715D12B4AE02411689E
:10673000F0220800104021420BD12849096811427B
:1067400009D12749274A11608021274A090211608F
:1067500001E03028F1D01A78012A0DD11D490968CD
:10676000090709D1F0201C4909680140402903D1DB
:106770001A490968014223D01B68DBB2012B25D1DD
:10678000144B1B681B0721D1134B1A68F0231A40C6
:10679000A02A04D1114A12681A4203D016E0D02A66
:1067A00014D1F7E7114B1A68012A03D1C022104B0C
:1067B0001A600BE00F4A1A601A68012AFCD1F5E74B
:1067C000C1218020C900C0054250D5E710BDC04698
:1067D000E00F00F0E40F00F0E80F00F0EC0F00F025
:1067E000DFFF07C004050040186C004000EC0640C5
:1067F00014EC0640759300000120704710B5036843
:106800001322DB69984710BD704700000369054AF1
:106810009950FC331A6A002AFCD0002201201A6227
:106820007047C0461C050000030010B55C331A78A1
:106830001F2313400122110099400D4B0424D967F6
:10684000C221036989005C505A60DA60A0220021ED
:10685000D20099500122074952425A500649143039
:106860005A500C395A5008315A50FFF703FF10BDE7
:1068700004E100E00C0500001405000010B5143020
:10688000FFF70AFF10BD10B51430FFF70BFF10BD66
:1068900010B51430FFF7F2FE10BD0000030070B514
:1068A0005E331C780269604BD45003005D331C7862
:1068B0005E4BD450030061331C785D4B012C0CD12E
:1068C00005005F352E78A225ED0056510500603594
:1068D0002E78A125ED00565100E00024D4509623D7
:1068E000DB00994238D996231B01994237D9962368
:1068F0005B01994236D996239B01994234D9E12311
:106900009B01994232D99623DB01994231D9E12387
:10691000DB0199422FD996231B0299422DD9E123FD
:106920001B0299422BD996235B02994229D9E12374
:106930005B02994227D9E1239B02994225D93D4B1D
:10694000994224D9E123DB02994223D9E1231B0395
:10695000994221D8384B21E09E23DB021EE09D2383
:106960001B031BE0354B19E0354B17E0EC239B0371
:1069700014E0344B12E0344B10E0344B0EE0344B57
:106980000CE0344B0AE0344B08E0344B06E0802343
:10699000DB0403E0324B01E080235B053149002436
:1069A00053500423243953501100FC31CC600C6245
:1069B000C1210134890014605C3094605350037825
:1069C0001F202200D9B20840824080342648FF347C
:1069D0005BB20251002B13DA0F230B40083B234C10
:1069E0009B089B001B1903242140A140FC348C40D0
:1069F000DD69A543C0248C4021002943D96111E001
:106A0000194C9B089B001B1903242140A140C02561
:106A1000FC348C40AD005E59A643C0248C4021005C
:106A200031435951026070BD0C050000140500008F
:106A30006C05000090D0030000D0BE0E00B0130023
:106A40000050270000A04E0000F0750000509D008F
:106A500000F0EB0000903A0100E0D70100B0AF0376
:106A600000705F072405000000E100E000ED00E099
:106A7000F7B5009308AB1B7800250193FA230400B7
:106A80009B0083600E4B45600833036014300F0099
:106A90001600FFF7D9FD23005C3327611E70009BB1
:106AA000084A9B00995823005D331970019B200010
:106AB0009B009A5823005E33DD701A70FEBDC046FD
:106AC00070B0000000AE0000036910B51A00FC327F
:106AD000D2680400002A0AD0A322D20099581430A8
:106AE000C9B2FFF7BCFD00222369FC33DA6010BD98
:106AF00010B50248FFF7E8FF10BDC04604120020A1
:106B0000162307B5022200930249013B0248FFF712
:106B1000AFFF07BD002000400412002070470000B6
:106B200010B500F011F8FFF7F9FF012000F0F0F9BF
:106B3000FEF700F9FEF712F9024B002BFAD000E045
:106B400000BFF7E700000000C421114A8900505837
:106B5000104B0340C020000203435350802391395F
:106B60009B02FF39535013608023A3220021DB05D1
:106B7000D20099500122A1209A60074BC000195001
:106B8000C120023180001950403019501A607047FE
:106B900000E100E0FF00FFFF00100140014B186022
:106BA0007047C046E8010020F7B50023202877D8B9
:106BB0003C4B8000C258042A14D006D8022A0DD0BB
:106BC0000ED80423012A14D069E0062A0ED00BD374
:106BD0001A2A0DD002231B2A0BD060E0082308E0FC
:106BE000102306E0202304E0402302E0802300E09D
:106BF00001232D4A1268082A04D9092A05D00A213E
:106C0000022404E00821002401E011000124A02551
:106C100001261C272548ED004651254D254E2D689F
:106C20001B02AD003D400195234D2D68009585590F
:106C3000AC466746214D3D401D4385518359C025D3
:106C40009C46009BAD021D40FF2367461B023B4054
:106C50002B43019D1D43009B5F0160231F402B00C0
:106C60003B431C4301238451154C036063680F4868
:106C7000002BFBD00024124B01255C60A123DB001C
:106C8000C3584560A025ED0044511BB2914207D086
:106C900002D98A1AD34003E0521A934000E000233D
:106CA0001800FEBD00AE0000EC01002000700040A6
:106CB000E401002004050000E0010020FF00FFFFC8
:106CC000FC700040F0B520286CD8374B8000C258CB
:106CD000364B1E68002E2ED1C2243548A400075919
:106CE000344B03253B40C0273F023B4303518023E5
:106CF000893C9B00FF3C03512F4F03602F4B803C8E
:106D0000D859FF3CA043D8510437D859A843204351
:106D1000D8510837D8590C35A843083D2843D851D5
:106D2000A820C0001E508026C120760280001E5080
:106D30001C601E4B1C6000231426214834005C4359
:106D4000255804006F1C0FD1142058432250A02056
:106D50000325C132FF329200C0051550194A0800C0
:106D60001268082A03D10BE0AA4218D1ECE7082ADE
:106D700002D9083AD14002E00820821A9140080066
:106D800014225343E3189A680C495132FF3292009F
:106D900058605050DA68C1239B00CA5002E00133AA
:106DA000032BCBD1F0BDC04600AE0000681200201E
:106DB00000E100E0FF00FFFF04050000009000403C
:106DC000F0010020E80100201E4BF0B5596C1800BE
:106DD0001D4A002914D0A025A12600230124ED0579
:106DE000F600D1584F1C06D0D7187F68002F02D06C
:106DF00027008F40AF5114333C2BF2D10023436462
:106E0000131DA02540329446002001240F4EED05AD
:106E1000DA680F49920057180A495218526C002A32
:106E20000CD01A1F1268511C05D01968FF2902D016
:106E300021009140A9513A00FC32506414339C4522
:106E4000E6D1F0BDFC900040F00100200C050000F0
:106E50000090004000B5202816D80C4A83009B58AB
:106E6000032911D8A0220800C133FF33D2059B00AB
:106E700000F06CF802080406002104E00C2102E096
:106E8000042100E00321D15000BDC04600AE000047
:106E900020280DD8074B8000C058A0220123D2051E
:106EA0008340002901D1044901E0A121C9005350C8
:106EB0007047C04600AE00000C0500000300002033
:106EC000202B0AD8A222A021D200C9058858034A43
:106ED0009B009B58D84001231840704700AE00002B
:106EE000084A0949094B10B51B688858FA22190A43
:106EF0001B0618439200002300F0F4F94904C00B6C
:106F0000084310BD04050000001001406C12002071
:106F100070B5041E09D0FFF7E3FF050000F014F878
:106F2000FFF7DEFF401B8442F8D870BD0022044BFF
:106F30009A60044A13680133DBB213607047C0469D
:106F4000FC1001406C1200207047000002B4714632
:106F500049084900095C49008E4402BC7047C0469C
:106F6000002243088B4274D303098B425FD3030A88
:106F70008B4244D3030B8B4228D3030C8B420DD39B
:106F8000FF22090212BA030C8B4202D31212090229
:106F900065D0030B8B4219D300E0090AC30B8B4267
:106FA00001D3CB03C01A5241830B8B4201D38B0315
:106FB000C01A5241430B8B4201D34B03C01A5241BA
:106FC000030B8B4201D30B03C01A5241C30A8B42FD
:106FD00001D3CB02C01A5241830A8B4201D38B02E8
:106FE000C01A5241430A8B4201D34B02C01A52418C
:106FF000030A8B4201D30B02C01A5241CDD2C309FE
:107000008B4201D3CB01C01A524183098B4201D379
:107010008B01C01A524143098B4201D34B01C01A64
:10702000524103098B4201D30B01C01A5241C308DC
:107030008B4201D3CB00C01A524183088B4201D34B
:107040008B00C01A524143088B4201D34B00C01A37
:107050005241411A00D20146524110467047FFE7A3
:1070600001B5002000F0F0F802BDC0460029F7D0BD
:1070700076E7704703460B437FD4002243088B42D8
:1070800074D303098B425FD3030A8B4244D3030BAF
:107090008B4228D3030C8B420DD3FF22090212BA74
:1070A000030C8B4202D31212090265D0030B8B42F0
:1070B00019D300E0090AC30B8B4201D3CB03C01ADA
:1070C0005241830B8B4201D38B03C01A5241430BB5
:1070D0008B4201D34B03C01A5241030B8B4201D3A5
:1070E0000B03C01A5241C30A8B4201D3CB02C01A10
:1070F0005241830A8B4201D38B02C01A5241430A88
:107100008B4201D34B02C01A5241030A8B4201D376
:107110000B02C01A5241CDD2C3098B4201D3CB011D
:10712000C01A524183098B4201D38B01C01A5241CC
:1071300043098B4201D34B01C01A524103098B42D0
:1071400001D30B01C01A5241C3088B4201D3CB00BB
:10715000C01A524183088B4201D38B00C01A52419E
:1071600043088B4201D34B00C01A5241411A00D24E
:1071700001465241104670475DE0CA0F00D04942B7
:10718000031000D34042534000229C4603098B4227
:107190002DD3030A8B4212D3FC22890112BA030AAF
:1071A0008B420CD3890192118B4208D38901921131
:1071B0008B4204D389013AD0921100E08909C309B6
:1071C0008B4201D3CB01C01A524183098B4201D3B8
:1071D0008B01C01A524143098B4201D34B01C01AA3
:1071E000524103098B4201D30B01C01A5241C3081B
:1071F0008B4201D3CB00C01A524183088B4201D38A
:107200008B00C01A5241D9D243088B4201D34B00A4
:10721000C01A5241411A00D20146634652415B10E6
:10722000104601D34042002B00D5494270476346C7
:107230005B1000D3404201B5002000F005F802BD0C
:107240000029F8D016E770477047C046D0400B1CA5
:107250001141203A03D49C461341184363465242DD
:10726000934018437047C0468446101C62468C46C3
:10727000191C634600E0C0461FB500F08BFD0028D6
:1072800001D40021C8421FBD10B500F0DFFC404210
:10729000013010BD10B500F07DFD002801DB00209D
:1072A00010BD012010BDC04610B500F073FD0028D0
:1072B00001DD002010BD012010BDC04610B500F05A
:1072C00005FD002801DC002010BD012010BDC046D6
:1072D00010B500F0FBFC002801DA002010BD0120F1
:1072E00010BDC046F0B54F464646C0B41604360C35
:1072F0009946330005042C0C070C150C63437E43A0
:107300006F4365431C0CAD1964199C46A64203D912
:1073100080235B02984647446346250CEF191D0401
:107320004B464A4343432D0C240464199918C91948
:1073300020000CBC90469946F0BDC046F0B55746BB
:107340004E4645464300E0B446028846760A1F0E84
:10735000C40F002F47D0FF2F25D0002380259A4649
:107360009946F600ED042E437F3F434642465D02B8
:10737000D20F5B006D0A1B0E904640D0FF2B39D018
:1073800080220020ED00D20415437F3BFB184246CB
:107390005746591C62408C4607430F2F5CD86F49F3
:1073A000BF00C9598F46002E45D108239A46063B97
:1073B0009946DAE7424602282DD0032800D1C3E0DF
:1073C000012800D0A2E0002500260240D4B27602B7
:1073D000ED05760A2E43E407264330001CBC904698
:1073E0009946A246F0BD002E1AD104239A46033BCB
:1073F0009946BAE72A00511E8A41901CC6E701202F
:10740000002DC3D0280001F0C9FB431F76309D40FA
:1074100043420020BAE70124FF2514400026D6E7A6
:10742000300001F0BBFB431F9E40002376304742F3
:107430009A46994699E70C239A46093B994694E760
:1074400080260024F603FF25C1E735004846B2E751
:10745000350022004846AEE72904090C0800370C25
:107460003604360C2C0C7943704367437443060C86
:1074700064183619B14203D980214902884647442D
:107480000004000C310409188D01681E8541890E25
:107490002943350CED19AD010D43290104D5012314
:1074A00069081D4063460D4319007F31002925DD21
:1074B000680704D00F202840042800D00435280194
:1074C00003D5274980330D401900FE29A3DC012490
:1074D000AD016E0A1440CDB279E78020C0030642A8
:1074E00007D0054205D128434602760A4446FF25C7
:1074F0006DE706437602760AFF2568E70124611AE4
:107500001B2905DD14400025002660E76346CBE714
:107510002E002023CE40591A8D406B1E9D412E43D4
:10752000730704D00F233340042B00D004367301BB
:1075300004D5012401251440002648E70124B601A2
:10754000760A1440002542E780260124F6032E43E4
:107550007602760A1440FF2539E7C046A0B0000045
:10756000FFFFFFF770B5002830D0C317C5185D4086
:10757000C40F280001F012FB9E231B1A962B0DDC72
:107580009622D21A95406A02520AD8B25202C00517
:10759000520AE40702432243100070BD992B19DC04
:1075A0009922D21A9540124A2A40690704D00F2125
:1075B0000D40042D00D00432510103D50C4B1A406C
:1075C0009F231B1A9201520AD8B2DFE70024002041
:1075D0000022DBE705222E00121AB921D6402A002C
:1075E000C91A8A40551EAA4135001543DBE7C0463B
:1075F000FFFFFFFBF8B556465F464D464446F0B4E4
:107600000F00FD0FAA4609037C002E005F00450F06
:10761000490A7F0D2943C5001803BC46400A570F8D
:10762000640DDB0F3843D2009A4500D1AAE06646CC
:10763000A61B002E00DCFFE06346002B39D10300BF
:10764000134300D0D9E06B0709D00F232B40042B44
:1076500005D02B1DAB42AD416D4249191D000B02F7
:1076600000D482E0CA4B01349C4200D1FEE00A0003
:107670005646C84BED081A405007640552020543B0
:10768000120B640D002112030B0D1B056405120B78
:107690001A436308C04CF60714401C436400640896
:1076A0003443280021003CBC90469946A246AB4694
:1076B000F8BDB74B9C42C6D080231B041843382E1C
:1076C00000DDEBE01F2E00DD1EE120239B1B9C460E
:1076D00003006746BB40984613004746F3403B43D0
:1076E0006746BA40571EBA4113430200F240EB1AF4
:1076F0009D42B6411D008A1A7642911B0B0231D57C
:107700004A02560A002E00D1B4E0300001F046FAD9
:107710000300083B1F2B00DDB5E020222900D21A10
:10772000D1409E400A009D4032439C4200DDB1E0C2
:107730001C1B631C1F2B00DDD5E02021140028003A
:10774000C91A8C40D8408D400443DA40681E8541F8
:1077500011002543002476E74146314300D134E24D
:10776000310045466B0700D06FE756464807ED08E5
:10777000C9080543864B9C4235D00A036405120BA9
:10778000640D7FE76346E31A9B46002B00DC8BE029
:107790006746002F3CD07E4FBC4200D153E7802784
:1077A0003F0438435B46382B00DCF7E00243501EB1
:1077B00082410020D2B253194218AB4289411D00C8
:1077C000494289180B02CDD5714B01349C4200D13E
:1077D0003DE101206F4A6B080A4028401843D50755
:1077E000054351082FE72B000B4300D1CBE1802349
:1077F0001B030B431A03120B44E7013E002E6DD10D
:10780000AE1AB5429B41091A5B42C91A350075E7A9
:107810000700174300D116E701235B429C46E3446F
:107820005B46002B00D0E0E0AA18AA429B41091851
:107830005B4259181500C5E7002E75D1661C760508
:10784000760D012E00DCF3E0AE1AB0464545BF418F
:107850000E1A7F42F61B370200D48FE0551BAA4256
:10786000B641411A76428E1B9A464BE75646002295
:10787000002507E7280001F091F920300300083BBC
:107880001F2B00DC49E72A002838824000259C4253
:1078900000DC4DE73F49E41A1140D4E60243501E94
:1078A0008241D3B2002222E7002B00D0F3E0631C18
:1078B0009C465B055B0D012B00DC9FE0344B9C4537
:1078C00000D1C3E0AA180918AA42804140424118D9
:1078D000CD075208154349086446B4E62C4B9C4238
:1078E00000D0ECE6AFE611001F3CE1400C00202B7D
:1078F00000D17FE04021CB1A9A4015436A1E954182
:107900000021254300242DE733000700203BDF4002
:107910003B00202E70D04027BE1BB0400243501EBB
:10792000824113430022E2E6002C4FD0184CA445BC
:1079300000D1ABE08024240476422143382E00DDC0
:10794000DFE01F2E00DD43E12027BC1BA1460C0019
:107950004F46BC40A0462C004746F4403C434F46AF
:10796000BD406F1EBD41F1402C43151BAA42924100
:10797000411A5242891A64469A46BFE64146454634
:10798000314300D0BEE6002600240025F2E6C046C2
:10799000FF070000FFFF7FFFFFFF0F801F2B59DC59
:1079A0002027FF1ABC46070063469F405B46B94646
:1079B0001700DF40B8464F4643461F4363469A4090
:1079C000531E9A415B463A43D840F4E60C002C43E0
:1079D0005CD0F643002E55D1551BAA42A441411A52
:1079E0006442091B9A46644688E6964FBC4200D022
:1079F000D8E628E6002280E700208FE70B002B4323
:107A0000002C00D0C2E0002B00D101E103001343A1
:107A100000D118E6AB18AB42B6410918764271188E
:107A20000A0200D409E1884A1D00114064460AE6B2
:107A3000002C5BD10E002E4300D08AE001001143E0
:107A400000D1C2E0010015009A46FCE56446002121
:107A500000258FE620235B429C46DC4463460700FA
:107A6000DF405B46BC46202B00D1ACE040235F46A4
:107A7000DB1B98400243501E8241634613431A00A9
:107A8000002098E66F4CA44500D057E70100150090
:107A900064469A46D7E5002C39D10C002C436ED0B1
:107AA000DB43002B1AD0674CA44568D0382B00DD8F
:107AB000A4E01F2B00DDAEE020240F00E41AA74055
:107AC000B9462F00DF40B846A3464F4644462743F9
:107AD0005C46A5406C1EA541D9403D43AD1895427A
:107AE0009B4109185B42591864466BE60C002C4315
:107AF00015D1010011437BD0010015009A46514C6D
:107B0000A1E50D43691E8D410021ECB22DE74D4CDE
:107B1000A44534D0802424045B422143C6E70400FA
:107B200014434ED0ED084C072C438025C9082D0383
:107B3000294208D0C6082E4205D1D2084107114378
:107B40000C009A463100620FC900E50011433D4C1C
:107B500079E50600164300D175E5AE1AB0464545F5
:107B6000BF410E1A7F42F61B370200D4F4E5551BC5
:107B7000AA42B641411A7642891B9A4663E5010042
:107B8000150064465FE5002200257BE5002B3BD015
:107B90000300134315D0ED084B072B438025C9087C
:107BA0002D03294207D0C4082C4204D141070B0001
:107BB0002100D2081343C9005A0F1143DD00214CA4
:107BC00041E5204C3FE5002054E700260025D1E5A3
:107BD00034000F00203CE7403C00202E2BD04027F3
:107BE000BE1BB1400D43691E8D4100212C43BCE6F4
:107BF000802100260903134C0025BBE50D43691EB7
:107C00008D410021EDB269E7010015000D4C1AE528
:107C10000100150017E51C000F00203CE7403C0068
:107C2000202B0CD04027FB1A99400D43691E8D4133
:107C30000021254352E70021D4E71D0092E50021F1
:107C4000F3E7C046FF070000FFFF7FFFF0B55F4688
:107C500056464D464446F0B41F035C00DB0F9A467F
:107C6000194B0E034D00C90F8046360B6D0D8B4628
:107C700091463F0B640D9D4219D0134B9C421BD083
:107C80000123A54206D018003CBC90469946A24666
:107C9000AB46F0BDBE42F6D1C845F4D1D34510D0B5
:107CA000002DF0D1304303005A1E9341EBE7310021
:107CB00001230143E7D1E0E73A430123002AE2D15F
:107CC000DEE70023DFE7C046FF070000F0B55F46B0
:107CD000444656464D46F0B41F033C0B2C4F0E0352
:107CE0004D00A3465C008446360B6D0DC90F9046CF
:107CF000640DDB0FBD422BD0254FBC422ED0002D92
:107D00000ED130430700814678427841002C17D1CC
:107D10005F463A4314D14B460020002B0AD006E0C0
:107D2000002C02D15846024301D099421AD00123B7
:107D3000484218433CBC90469946A246AB46F0BD2B
:107D40000028F2D058425841012240421043F1E746
:107D500037000743D0D002204042EBE75F4617438D
:107D6000CDD0F8E7A542E2DC05DB5E45DFD808D0E0
:107D700000205E45DED2484248410123404218437C
:107D8000D8E7C445D3D80020C445F4D3D2E7C046D1
:107D9000FF070000F0B55F464D4644465646F0B436
:107DA0001C03240BA4462F4C0F034D005E00C90F8B
:107DB00080463F0B6D0D8B469146760DDB0FA5423D
:107DC00020D0284CA64222D0002D12D13843444264
:107DD0004441002E20D0002C0DD05C426341012490
:107DE0005B421C4320003CBC90469946A246AB46F1
:107DF000F0BD002E17D05B4519D05B465C420123D5
:107E00001C43EFE7390002240143EBD1D9E7614677
:107E100002241143E6D1D7E761460A43DBD10024AF
:107E20000028DFD0E9E761460A43E4D1E5E7B5423F
:107E300003DD01225C421443D4E7B542CDDB674544
:107E4000DBD809D000246745CCD259464C42614169
:107E5000012449420C43C5E7C845CED80024C84593
:107E6000F3D3BFE7FF070000F0B55F4656464D4627
:107E70004446F0B40D0399464E002B0B87B0070023
:107E8000924680469B46760DCC0F002E69D06D4BF6
:107E90009E4235D05B468022DD001204430F13431F
:107EA0002B439B46C3009846674B00279C46002304
:107EB000664401934A4615035000D20F53462D0BDA
:107EC000400D914600D176E05E4A90426CD080220F
:107ED0005B0F120413435C4AED0094461D43534666
:107EE0000022DB00604449463618701C6140029055
:107EF00017430F2F00D9AFE05448BF00C759BF4602
:107F00005B461F4300D088E000239B46984602331F
:107F100008270193CEE74946022A6AD0032A00D1F6
:107F200009E2012A00D0BBE1114000220023002514
:107F30009046CCB200212D030A0D12052D0B1543DE
:107F4000434A1B0515401D436D00E4076D0825439A
:107F50004046290007B03CBC90469946A246AB4635
:107F6000F0BD034352D05B46002B00D18AE1584656
:107F700000F014FE03000B3B1C2B00DD7BE11D22F7
:107F8000D31A3A0001005D46DA4008398D401300EB
:107F90008F402B439B46B8462E4B00279C46002320
:107FA00060444642019385E752462A432CD100257E
:107FB0000023022297E752462A4321D0002D00D108
:107FC00054E1280000F0EAFD03000B3B1C2B00DD10
:107FD00046E11D21CB1A51460200D9405346083ACA
:107FE000954093400D431B4A944660444042002212
:107FF00079E7012400220C40124B0025904699E7B6
:108000000025002301226EE703226CE700239B4634
:1080100098460133042701934CE703230C2701936F
:1080200048E700238025984600242D03054B81E76F
:108030005D464346019A6FE75D4643462100019A3B
:108040006AE7C046FF07000001FCFFFFE0B0000048
:10805000FFFF0F80F30300004246120C91461A0CFA
:108060009446424617044A461B041B0C5A4360467A
:1080700090464A4642431000039262461C003F0C61
:108080007A437C4342440192220C9246019A524424
:10809000904506D98246802040028046C244504620
:1080A0000390100C049048462404240C1204121966
:1080B00005922A0C2D042D0C68432C00824648465C
:1080C0007C4350438146200C8046574357444744E5
:1080D000BA4503D9802040028046C144380C3F0491
:1080E000B84648442404240C01900498A044404419
:1080F00004905846000C814658460404200C8246E1
:10810000070048465F434C4643436046604364462D
:10811000834650464443380C8446E4186444A342E2
:1081200003D980235B029C46E34448463F04230C6A
:108130003F0C2404E419574668436F4384464D4678
:10814000504655434243380C814662444A445B449E
:10815000944503D9802040028446654403983F0437
:10816000834604983F0C8446E344C3458041404223
:108170008246100484460198674484466744A344B9
:10818000BC46A345A4419946D44464428742BF41BA
:10819000D4458041E144A04699459B417F424042FD
:1081A000C8440743120CBA18A045A4415F423B00E3
:1081B00064422343D71843467D19DB0D6D021D43EE
:1081C0005B465A02059B1A43531E9A415B46DB0DE0
:1081D0001A4343465B021343EA0107D501225C08B8
:1081E00013402343EA07029E13436D08574AB2180F
:1081F000002A4BDD580709D00F201840042805D06D
:10820000181D98429B415B42ED180300E80104D51C
:108210004F4A15408022D200B2184E48824200DDFB
:10822000E7E60124DB08680718436D025305804622
:108230002D0B5B0D0C407DE6802259461203114246
:1082400008D0154206D115432D0398462D0B4C46F8
:10825000414B6FE65D4615432D032D0B3E4B69E602
:1082600003005546283B9D400023BCE6504600F0E5
:1082700095FC2030A8E60300283B9F400023BB4626
:10828000984689E600F08AFC203073E60124A61A9D
:10829000382E07DD00220C4000230025904649E6D9
:1082A000029EA3E71F2E20DC20222C001800921B28
:1082B000F040944093400443581E83411C43F540D2
:1082C000630709D00F232340042B05D023001C1D76
:1082D0009C4292415242AD182B021FD5012400222C
:1082E0000C4001230025904624E61F202C0040422C
:1082F000821AD440202E1CD04022961BB5402B431E
:10830000581E83410720234318400025002809D028
:108310000F2200251A401C00042AD8D12300680728
:108320006D022D0B0124DB08034398460C4000230B
:1083300000E60025E3E780220124120315432D0304
:1083400098462D0B0C40044BF4E5C046FF0300009B
:10835000FFFFFFFEFE070000FF070000F0B55746D5
:108360004E464546E0B40E001100F20F9246C5009D
:10837000420F180337037400400A4E0F7F0A304340
:10838000CF4E17435A00640D520DDB0FC900B242A5
:1083900000D1E5E001267340A61AB446534500D14A
:1083A000AFE0002E00DC0DE1002A3AD103000B43C0
:1083B00000D0E4E06B0709D00F232B40042B05D03D
:1083C0002B1DAB42AD416D427F191D003B0200D415
:1083D00088E0BB4B01349C4200D110E13A00B94B1C
:1083E00051461A4001235007ED0852026405054327
:1083F000120B640D0B400021280012030D0D120B0F
:1084000064052D0515436208AF4CDB072C4014436F
:10841000640064081C4321001CBC90469946A24697
:10842000F0BDA74B9C42C5D080231B041843634674
:10843000382B00DDFDE01F2B00DD30E162462023FC
:108440009B1A02009A40664690460A009940F24004
:1084500046464B1E99413243114363460200DA40BF
:10846000691A8D429B410D00BA1A5B42D71A3B0232
:1084700035D57A02530A98464346002B00D1C4E012
:10848000404600F08BFB0300083B1F2B00DDC5E0DE
:1084900020222900D21A4746D1409F400A009D4021
:1084A0003A439C4200DDC0E01C1B631C1F2B00DD17
:1084B000E4E0202114002800C91AD8408C408D40E7
:1084C0000443DA40681E854117002543002471E704
:1084D000424663461A4300D14CE2674645466B0765
:1084E00000D069E7012351467807ED08FA080B40F0
:1084F000054373498C4238D012036405120B640D96
:1085000079E7002E00DC9AE0002A47D06C4A9442BA
:1085100000D14FE78022120410436246382A00DC63
:1085200008E10143481E81410022C9B24919D2190C
:10853000A942BF410D007F42BF183A0200D442E178
:108540005F4A0134944200D14EE101205D4A69083E
:108550003A4028400843D507054357089A4629E77B
:1085600006000E4300D017E714E72900114300D19D
:10857000F9E1802109030A431203120B3BE70123AF
:108580005B429846C4446346002B72D1691A8D42FF
:108590009B413F1A5B42FF1A0D0068E702000A4345
:1085A00000D107E7012252429046C4446246002AA5
:1085B00000D0E6E06918A942B6413F187642F719A3
:1085C0000D00BAE7002E00D080E0621C5205520D6B
:1085D000012A00DCF9E06A1A91464D45B6413A1A83
:1085E0007642921B9046120200D499E04D1BA9429C
:1085F0008941C71B49427A1A90469A463CE752463F
:108600000123002513400022F5E6280000F0C6FAF9
:1086100020300300083B1F2B00DC39E72A002838F4
:10862000824000259C4200DC3EE7264FE41A1740BA
:10863000C0E60143481E81410022C9B210E7002E66
:1086400000D0F1E0621C94465205520D012A00DC74
:10865000A0E01B4A944500D1C5E06918A9429241A7
:108660003F185242D2194908D5070D4357086446AE
:10867000A0E6134B9C4200D0D9E69BE611001F3CBC
:10868000E1400C00202B00D180E04021CB1A9A4021
:1086900015436A1E95410027254300241FE76346C2
:1086A0000200203BDA406346202B71D0402366460F
:1086B0009B1B98400143481E814111430022CFE695
:1086C000FF070000FFFF7FFFFFFF0F80002C48D057
:1086D000CA4CA24200D1A2E07442A14680242404E4
:1086E00027434C46382C00DDDBE01F2C00DD44E145
:1086F0004E462024A41B3E00A640A246B0464C464F
:108700002E00E640B4464646644626435446A540FD
:108710006C1EA54134002C434D46EF400D1B28E054
:108720004A4643464D461A4300D0A5E6002300249E
:108730000025DEE61F2A5ADC66462022921B060030
:1087400096409146B04662460E00D64042461643D9
:108750004A4691404A1E9141020060463143C24060
:10876000E4E63C002C435AD0F443A146002C52D1FD
:108770004D1BA9428941C71B49427F1A14009A46E2
:1087800075E69E4A944200D0C7E613E600227FE7D2
:1087900000208FE7002C00D0C8E03B002B4300D125
:1087A0000FE103000B4300D104E66918A9429B4185
:1087B0003F185B42DF193B0200D41AE1904B0D00D9
:1087C0001F406446F6E59A4689E63A002A43002CA3
:1087D0005CD1002A75D102000A4300D1CAE007002B
:1087E0000D009A46E6E564460022002581E66246D1
:1087F0000600203AD6406246B046202A00D1B7E0B3
:1088000040226646921B904001434246481E8141E9
:10881000114300228AE6794CA24200D061E70700AA
:108820000D0014009A46C5E5002C41D13C002C43B4
:1088300078D0F443A146002C20D0704CA24271D0D5
:108840004C46382C00DDB2E01F2C00DDBCE02026B9
:10885000341BA2463C005646B4404E46A0462C006F
:10886000F440A446444666463443A4465446A540D4
:1088700064466E1EB54125434C46E7406D188D4257
:1088800089413F184942CF19140056E6002A2FD1DA
:1088900002000A4300D184E007000D009A46574CBD
:1088A00088E53D436F1EBD41ECB200270D1B60E71C
:1088B000524CA24236D0744280263604A146374339
:1088C000BEE702000A4300D174E56A1A90464545A6
:1088D000B6413A1A7642921B9446120200D4F7E54A
:1088E0004D1BA9428941C71B49427F1A9A4661E53F
:1088F00002000A433AD0ED087C072C438025FA0891
:108900002D032A4208D0C7082F4205D145072C0065
:108910003A009A46C9080C43670FD200E500174396
:10892000364C47E507000D00140043E53A002A43A2
:1089300043D002000A4319D0ED087C072C43802560
:10894000FA082D032A4207D0C6082E4204D1470751
:108950003C003200C9080C43D700620FE500174302
:108960009A46264C26E50022002544E5234C21E5C5
:10897000002049E700230025BBE54C463E00203C93
:10898000E6404C46B446202C31D040244E46A61B2F
:10899000B7403D436C1EA54164462C4300270D1B88
:1089A000E7E6802200231203144C0025A1E53D4395
:1089B0006F1EBD410027EDB260E707000D000F4CB0
:1089C000F8E407000D00F5E44E463C00203EF4407C
:1089D000A0464C46202C0ED040244E46A41BA74057
:1089E0003D436F1EBD4144460027254346E700270F
:1089F000CFE70D0073E50027F2E7C046FF07000050
:108A0000FFFF7FFF0B0330B5134D1A0B4B005B0DBF
:108A1000C90F0024AB4211DD104CA34210DC8024AE
:108A2000640322430E4CE41A1F2C0CDD0D48C31ABC
:108A3000DA4013005C42002900D11C00200030BD48
:108A4000094BCC18FAE7E040084CA44663449A402E
:108A500013000343EEE7C046FE0300001D040000C0
:108A60003304000013040000FFFFFF7FEDFBFFFF56
:108A700070B5002830D0C317C4185C40C50F200063
:108A800000F08CF8174B184A1B1AD21A1F2A18DD4F
:108A9000164AD21A9440002224035B05240B5B0D76
:108AA0000021100024030A0D1205240B1443104A60
:108AB0001B0514401C436400ED0764082C4321008F
:108AC00070BD210091400A000B21081AC4405B05CB
:108AD0002403240B5B0DE3E7002500230024002280
:108AE000DEE7C0461E04000033040000130400004B
:108AF000FFFF0F804200120E511C4302C9B270B535
:108B00005D0AC40F012915DDE02189008C466D073F
:108B10001B0B6244002128000D0D2D052B431C4D1D
:108B200052052B40520813435B00E4075B082343C4
:108B3000190070BD002A15D1002D1FD0280000F0AB
:108B40002DF80A281DDC0B232A001B1ADA4013001B
:108B50000200153295400F4A1B03121A52051B0BD7
:108B6000520DD7E7002D06D080221B0B12031343B2
:108B70006D07094ACEE7084A0023CBE7002200230D
:108B8000C8E703000B3B9D402B000025E3E7C046F0
:108B9000FFFF0F8089030000FF0700001C21012355
:108BA0001B04984201D3000C10391B0A984201D3D0
:108BB000000A08391B09984201D30009043902A2AE
:108BC000105C40187047C046040302020101010115
:108BD00000000000000000007FB51D000A4B0600E9
:108BE0001B68D868002A02D1084C230001E013005A
:108BF000074C0293009133002A000649019400F0CB
:108C000021F800F023FEC0468C020020A6AA000036
:108C100020B100002DB10000084B10B50400002B5E
:108C200002D0002100E000BF054B1868836A002BCA
:108C300000D09847200001F0F3FAC0460000000081
:108C400060B100000EB403B5010003AB044804CBCF
:108C50000068019300F016F902B008BC03B0184791
:108C60008C0200200E4B70B500251E000D4CE41A3E
:108C7000A410A54204D0AB00F35898470135F8E79B
:108C800001F0D0FA084B00251E00084CE41AA4108D
:108C9000A54204D0AB00F35898470135F8E770BD02
:108CA000940200209402002094020020A4020020DC
:108CB00010B5034B0100186800F066F810BDC046FF
:108CC0008C02002010B5034B0100186800F016F864
:108CD00010BDC0468C020020002310B59A4203D07C
:108CE000CC5CC4540133F9E710BD030082189342F1
:108CF00002D019700133FAE77047000030B500293F
:108D00003ED004390B68002B00DAC9181D4A1368DD
:108D10001400002B02D14B60116031E08B420DD961
:108D20000A688818834203D118685B6882180A6051
:108D30004B60216024E08A4203D813005A68002A5D
:108D4000F9D11D685C198C420BD109686918581853
:108D50001960824214D110685268411819605A6033
:108D60000EE08C4202D90C23036009E008680C185D
:108D7000A24203D114685268201808604A60596002
:108D800030BDC04674120020032370B5CD1C9D4336
:108D9000083506000C2D01D20C2505E0002D03DA64
:108DA0000C230020336040E0A942F9D81F4B1C6817
:108DB0001A002100002913D00B685B1B0DD40B2B6C
:108DC00002D90B60CC181EE08C4202D1636813609C
:108DD0001AE04B6863600C0016E00C004968E9E794
:108DE000134C2368002B03D1300000F033FB2060CC
:108DF0002900300000F02EFB431CD1D00323C41CFB
:108E00009C43A0420AD12560200007220B30231D7D
:108E10009043C31A09D05A42E25006E0211A3000AA
:108E200000F018FB431CEED1BAE770BD74120020AD
:108E300070120020936810B5013B9360002B05DA97
:108E40009469A34208DBCBB20A2B05D01368581CE7
:108E500010601970C8B201E000F02CFC10BDF8B52C
:108E600006000F001400D518AC4208D021783A0053
:108E70003000FFF7DFFF0134431CF5D100E0002094
:108E8000F8BD0000F0B59FB006000F0002920593F8
:108E9000002804D08369002B01D100F0D3FD7F4B63
:108EA0009F4201D1776808E07D4B9F4201D1B768AE
:108EB00003E07C4B9F4200D1F768BB891B070AD5B2
:108EC0003B69002B07D0002306AD6B6120336B7626
:108ED0001033AB763DE03900300000F043FC002851
:108EE000F1D001204042D6E0059A111D126805918B
:108EF000002A00DA7FE00992013423782E2B00D17A
:108F00008DE021780322684800F082FE002807D017
:108F1000654B2A68C01A4023834013432B600134F9
:108F20002178631C062261480293297600F070FEC6
:108F3000002800D19DE05E4B002B00D090E007227E
:108F4000059B07339343083305936B69039A9B187A
:108F50006B61029C2378002B04D1029BE31A0493DB
:108F600012D003E0252BF8D00134F3E7049B029ADA
:108F700039003000FFF773FF431C00D186E06A69B7
:108F8000049B944663446B612378002B7ED00122BE
:108F9000002352426A6002A95432521801342B60F5
:108FA000EB60AB601370AB6521780522414800F09F
:108FB0002FFE002808D03F4B2A68C01A01238340A7
:108FC00013432B600134EFE72B68DA0604D55322F4
:108FD000202102A8121811701A0704D553222B2140
:108FE00002A81218117022782A2A00D17CE7099B66
:108FF00000200A2105E05242EA60022213432B605E
:109000007AE72278303A092A04D84B4301349B1876
:109010000120F6E7002800D16FE709936DE7637838
:109020002A2B0AD1059B02341A1D1B680592002BBE
:1090300001DA01235B42079363E700230A201A0049
:1090400001346B6021783039092904D84243013456
:1090500052180123F6E7002B00D152E7079250E7A0
:1090600005AB00933A00144B2900300000E000BF2C
:1090700007E005AB00933A000F4B2900300000F0E9
:109080008BF80390039B013300D05EE7BB895B063E
:1090900000D526E70B981FB0F0BDC04698B200007F
:1090A000B8B20000D8B200006AB100006EB1000092
:1090B0000000000064B100005F8E0000F7B51700EB
:1090C00001938A680B6900900C00934200DA130048
:1090D00022003B6043321278002A01D001333B600A
:1090E00023689B0602D53B6802333B600625236854
:1090F0001D401ED0230043331B785A1E9341226823
:1091000092061CD53020E1184331087021005A1C0A
:1091100045310978A2184332023311700FE0220062
:109120000123193201990098089EB047431C0ED0C4
:109130000135E3683A689B1A9D42F0DBDAE72200CA
:10914000019943320098089DA847431C02D1012091
:10915000404220E006232068E1683A680340002589
:10916000042B03D18D1AEB43DB171D40A368226942
:10917000934201DD9B1AED180027BD420AD0220060
:1091800001231A3201990098089EB047431CDED093
:109190000137F2E70020FEBDF0B58BB006920A0061
:1091A00043320793059004920A7E0C00109B6E2AAE
:1091B00000D1ABE011D8632A22D009D8002A00D10F
:1091C000B5E0582A00D0C5E045310A70814A4FE029
:1091D000642A1DD0692A1BD0BCE0732A00D1AAE002
:1091E00009D86F2A29D0702A00D0B3E0202209685C
:1091F0000A43226037E0752A1FD0782A33D0A9E0CD
:109200000E001A684236111D196013683370A4E00D
:1092100021681A68080606D4490604D5111D19608C
:109220000023D55E02E0111D19601568002D3BDAA0
:109230002D23049A6D42137036E021681A680806DF
:1092400006D4490604D51568111D1960ADB202E0B7
:10925000111D196015685F4B227E039308276F2A42
:109260001DD00A271BE022007821453211705A4A8E
:1092700019680392081D226818600D68100602D450
:10928000500600D5ADB2D30702D520231A43226081
:109290001027002D03D1202322689A432260230047
:1092A000002243331A7002E00A274A4B0393636893
:1092B000A360002B09DB0422216891432160002D6B
:1092C00005D1049E002B11D07BE0002D79D0049EA7
:1092D00028003900FDF7CAFE039B013E5B5C2800B5
:1092E00033703900FDF73CFE051EF1D1082F09D17E
:1092F0002368DB0706D563682269934202DC3023CA
:10930000013E3370049B9B1B23612BE009681A68A4
:10931000080607D4490605D5111D19601368A28AED
:109320001A8004E0111D1960136862691A60002335
:10933000049E236116E01A68111D19601668002149
:109340006268300000F064FC002801D0801B60607F
:10935000636803E026004236327001232361002354
:10936000049A1370079B09AA00932100069B059895
:10937000FFF7A4FE431C02D10120404227E02369ED
:10938000320006990598079DA847431CF4D023682E
:1093900000259B070FD4099BE068984217DA180054
:1093A00015E022000123193206990598079EB0475F
:1093B000431CE1D00135E368099A9B1A9D42F0DB1A
:1093C000E9E72600039B42361B7833708EE70BB02B
:1093D000F0BDC04675B1000086B10000154B10B558
:1093E0001C68A36B002B15D11820FFF761FC124BF2
:1093F000A0630380114B01224380114B8380114BEA
:10940000C380114B038105234381063383810023ED
:1094100002614361A46B0D4A206961690C4BFDF741
:1094200061FF0122002380185941206161614800D9
:10943000400810BD8C0200200E330000CDABFFFFB2
:10944000341200006DE6FFFFECDEFFFF2D7F954C30
:109450002DF45158002370B5064C05000800236018
:1094600000F0C8FE431C03D12368002B00D02B6002
:1094700070BDC0468C2600200CB430B5164B9DB094
:109480000C1E1D6804DA8B2301202B6040421DE076
:10949000822302A99B008B810023029008619C42D9
:1094A00000D0631E8B604B6101235B42CB81209A0D
:1094B00021AB2800019300F053FC431C01DA8B23FD
:1094C0002B60002C02D00023029A13701DB030BC18
:1094D00008BC02B01847C0468C0200200EB410B57C
:1094E0009DB002A9029008610B48822488604861FF
:1094F000012040421FABC881084804CBA40000688B
:1095000001938C8100F02CFC0023029A13701DB093
:1095100010BC08BC03B01847FFFFFF7F8C0200207F
:1095200002780B78002A03D0013001319A42F7D03B
:10953000D01A7047031C0A7801311A700133002ACF
:10954000F9D170470023C25C0133002AFBD1581EB9
:109550007047030030B5002A0DD00C7801335D1E32
:10956000013A2C700131002CF5D19A189A4202D0A0
:109570001C700133FAE730BDF0B51E00454B87B0D3
:109580001B680192029308220B00059003911C783E
:1095900002995D1C09194878104001D02B00F6E7AC
:1095A0002D2C04D19D1C5C780123009304E00090D5
:1095B0002B2C01D15C789D1C002E02D0102E0AD1DC
:1095C00062E0302C5ED120222B789343582B54D16B
:1095D00010266C780235009F31007B1E9F412E4B78
:1095E000FF183800FDF742FD380004913100FDF707
:1095F000B7FC00230322070094461800029A1219B0
:1096000051780422114201D0303C07E062461140FB
:1096100017D03722012900D02032A41AA64210DD2B
:109620005A1C0BD0B84207D802D1049B9C4203DCE1
:1096300070430123201801E001235B422C7801359F
:10964000DCE75A1C0BD10098059A431E9841124B37
:10965000C01822231360019B002B0AD117E0009A47
:10966000002A00D04042019A002A10D0039A002B11
:1096700000D06A1E019B1A6009E03024002EAAD196
:109680000826A8E70A26A6E7302C9CD0A3E707B057
:10969000F0BDC04690020020FFFFFF7F10B5130011
:1096A0000A00010002480068FFF766FF10BDC046CF
:1096B0008C020020F8B505000F001400002804D02B
:1096C0008369002B01D100F0BDF9234B9C4201D1ED
:1096D0006C6808E0214B9C4201D1AC6803E0204B50
:1096E0009C4200D1EC68A369A360A3891B070AD53B
:1096F0002369002B07D023682269FEB2981A636998
:1097000098420FDB08E02100280000F02BF8002829
:10971000F1D0012040421DE02100280000F024F992
:109720000028F6D1A3680130013BA36023685A1CCE
:1097300022601F706369984205D0A3893000DB075F
:1097400008D50A2E06D12100280000F00DF90028C6
:10975000DFD13000F8BDC04698B20000B8B20000BA
:10976000D8B20000354B70B51D6806000C00002D06
:1097700005D0AB69002B02D1280000F063F9304B13
:109780009C4201D16C6808E02E4B9C4201D1AC6830
:1097900003E02D4B9C4200D1EC68A3899AB21107DB
:1097A00023D4D10607D40922012032603732134373
:1097B000A381404240E0530713D5616B002908D0D4
:1097C00023004433994202D03000FFF797FA002378
:1097D00063632422A3899343A381002363602369E5
:1097E00023600822A3891343A3812369002B0BD193
:1097F000A023A2899B00134080229200934203D0B1
:109800002100300000F0B2F90123A289134005D0F5
:109810000023A36063695B42A36103E0910700D466
:109820006369A36000202369834205D1130603D531
:1098300040231A43A281013870BDC0468C0200202B
:1098400098B20000B8B20000D8B2000010B50620EF
:1098500000F0AEFB012000F0E3FC0000F7B58A89C0
:1098600005000C0013075AD44B68002B02DC0B6C6C
:10987000002B19DDE76A002F16D000232E682B601D
:1098800080235B011A4001D0606D14E00123216A3E
:109890002800B847431C0ED12B68002B0BD01D2B82
:1098A00001D0162B02D12E6000205AE04022A3895D
:1098B0001343A38155E0A3895B0706D56368C01AEB
:1098C000636B002B01D0236CC01A00230200216AB5
:1098D0002800E76AB847A389421C06D129681D29D8
:1098E0003AD8204ACA40D20736D50022626022699F
:1098F0002260DB0405D5431C02D12B68002B00D16C
:109900006065616B2E600029CED0230044339942FC
:1099100002D02800FFF7F2F90020606321E00F6910
:10992000002FC1D00B680F60DB1B0193002392074F
:1099300000D14B69A36003E0019B3F181B1A019300
:10994000019B002BB0DD019B3A00216A2800A66A2A
:10995000B0470028F0DCA389402201201343A381F3
:109960004042FEBD010040200B6970B505000C00AF
:10997000002B01D100201CE0002804D08369002BBB
:1099800001D100F05FF80B4B9C4201D16C6808E0FC
:10999000094B9C4201D1AC6803E0084B9C4200D1CA
:1099A000EC680C22A35E002BE4D021002800FFF716
:1099B00055FF70BD98B20000B8B20000D8B20000E8
:1099C00010B5024900F0B0F810BDC046699900001A
:1099D000002310B504000360436083608181436607
:1099E000C281036143618361190008225C30FFF783
:1099F0007CF9054B24626362044BA362044BE3626F
:109A0000044B236310BDC046F19F000019A0000065
:109A100051A000007DA0000070B568254B1E5D437D
:109A20000E0029007431FFF7AFF9041E08D00021A1
:109A30002A00016046600C30A0606832FFF755F9DB
:109A4000200070BD836913B50400002B28D1836406
:109A5000C3640365134B144A1B68826201939842E6
:109A600001D101238361200000F020F86060200014
:109A700000F01CF8A060200000F018F80022E06060
:109A800004216068FFF7A4FF01220921A068FFF705
:109A90009FFF02221221E068FFF79AFF0123A361D2
:109AA00013BDC04660B10000C1990000F8B51D4B60
:109AB00006001D68AB69002B02D12800FFF7C2FF2A
:109AC0004835AC686B68013B05D40C22A75E002FBB
:109AD00010D06834F7E72B68002B01D02D68F0E731
:109AE00004213000FFF798FF28600028F6D10C23EE
:109AF000336016E0012320005B42E3810233A3813F
:109B000067662760A760676027616761A7615C304F
:109B100008223900FFF7E9F820006763A763A7640C
:109B2000E764F8BD60B10000F7B504000700002647
:109B300001914834002C16D06368A5680093009BFF
:109B4000013B00930DD4AB89012B08D90E22AB5EEB
:109B5000013304D029003800019B9847064368353B
:109B6000EDE72468E6E73000FEBD0000F0B58B8924
:109B700091B006000C009B0726D40E23C95E002975
:109B800004DA8023A5891D4010D10CE001AA00F061
:109B9000A1FA0028F5DBF023029D1B021D401A4BA1
:109BA000ED186B425D418027FF0001E00025402752
:109BB00039003000FFF7E8F800280CD1A3899A0596
:109BC0001FD402221343A381230047332360236160
:109BD0000123636115E080220C4BB362A3892060EE
:109BE0001343A38120616761002D0AD00E23E15E3B
:109BF000300000F081FA002803D00122A38913432A
:109C0000A38111B0F0BDC04600E0FFFFC199000084
:109C1000C9B28218904204D003788B4202D001303E
:109C2000F8E70020704710B5884202D98B18984297
:109C300001D3002305E09B1A013A08D3995C8154B3
:109C4000FAE7934203D0CC5CC4540133F9E710BD6A
:109C5000F8B506000C001500002904D11100FFF72B
:109C600093F8040018E0002A03D1FFF747F82C000E
:109C700012E000F067FA85420ED929003000FFF7A4
:109C800083F8071E07D021002A00FFF725F82100DE
:109C90003000FFF733F83C002000F8BDF0B58E68C7
:109CA00085B007000C00039201939E4243D8902395
:109CB0008A89DB001A423ED003250969236801988E
:109CC0005B1A029363695D43EB0F5D19029B6D1094
:109CD00001331B18AB4200D91D00530510D52900D4
:109CE0003800FFF751F8061E14D0029A2169FEF7DA
:109CF000F3FFA289194B134080221343A38112E082
:109D00002A003800FFF7A4FF061E0CD12169380095
:109D1000FEF7F4FF0C23402201203B60A389404260
:109D20001343A38117E0029B2661F6182660656144
:109D3000019EED1AA560019BB34200D21E003200C5
:109D400003992068FFF76FFF0020A3689B1BA360A7
:109D500023689E19266005B0F0BDC0467FFBFFFF5B
:109D6000F0B59FB0029005938B890F0016001B067B
:109D700010D50B69002B0DD14021FFF705F8386095
:109D80003861002804D10C23029A01381360D8E00E
:109D900040237B61002306AD6B6120336B7610336B
:109DA000AB7634002378002B03D1A31B049312D08D
:109DB00003E0252BF9D00134F4E7A31B320039006E
:109DC0000298FFF76BFF431C00D1B4E06A69049B63
:109DD000944663446B612378002B00D1ABE00122F1
:109DE000002352426A6002A95432521801342B6097
:109DF000EB60AB601370AB65534E217805223000E9
:109E0000FFF706FF002807D00123801B83402A6844
:109E1000013413432B60EFE72B68DA0604D5532295
:109E2000202102A8121811701A0704D553222B21E1
:109E300002A81218117022782A2A03D0099B002048
:109E40000A210EE0059A111D12680591002A01DB16
:109E5000099204E05242EA60022213432B6001346B
:109E60000BE02278303A092A04D84B4301349B187E
:109E70000120F6E7002800D0099323782E2B1ED16D
:109E800063782A2B0AD1059B02341A1D1B680592A0
:109E9000002B01DA01235B42079310E000230A2024
:109EA0001A0001346B6021783039092904D8424303
:109EB000013452180123F6E7002B00D00792234EFD
:109EC000217803223000FFF7A3FE002806D04023AC
:109ED000801B83402A68013413432B6021780622BB
:109EE0001B48661C2976FFF793FE002812D0194BF9
:109EF000002B06D10722059B0733934308330593B4
:109F000014E005AB00933A00134B2900029800E0DF
:109F100000BF07E005AB00933A000F4B2900029801
:109F2000FFF73AF90390039B013304D06B69039A5E
:109F30009B186B6135E7BB890B985B0601D5012047
:109F400040421FB0F0BDC04664B100006AB10000DD
:109F50006EB10000000000009D9C000070B5040080
:109F60000D1E1F2D04D916230360012040421EE060
:109F7000426C002A04D08B00D2181368002B08D141
:109F8000200000F031F82A000100200000F01AF84B
:109F90000DE00020012B0AD0591C03D11733236098
:109FA000013004E00024280014609847200070BDB0
:109FB00010B5034B01001868FFF7D0FF10BDC04675
:109FC0008C020020002370B5064C0500080011002B
:109FD000236000F0F7F8431C03D12368002B00D066
:109FE0002B6070BD8C26002010B500F0DBF810BD92
:109FF00070B50C000E25495F00F0B0F8002803DBB7
:10A00000636D1B18636503E0A289024B1340A381B3
:10A0100070BDC046FFEFFFFFF8B51F008B8905003C
:10A020000C001600DB0505D50E23C95E00220223B5
:10A0300000F074F8A289054B28001340A381320078
:10A040000E23E15E3B0000F01FF8F8BDFFEFFFFFBD
:10A0500070B50C000E25495F00F060F8A389421C22
:10A0600003D1054A1340A38104E080225201134327
:10A07000A381606570BDC046FFEFFFFF10B50E23E2
:10A08000C95E00F015F810BD70B50500080011009C
:10A090000022064C22601A0000F0BAF8431C03D1DB
:10A0A0002368002B00D02B6070BDC0468C2600209A
:10A0B000002370B5064C05000800236000F062F82C
:10A0C000431C03D12368002B00D02B6070BDC04619
:10A0D0008C260020002370B5064C050008001100F6
:10A0E000236000F057F8431C03D12368002B00D0F5
:10A0F0002B6070BD8C260020002370B5064C050037
:10A100000800236000F056F8431C03D12368002B9D
:10A1100000D02B6070BDC0468C26002070B50500B5
:10A12000080011000022064C22601A0000F052F8CC
:10A13000431C03D12368002B00D02B6070BDC046A8
:10A140008C2600200B1F1A68101F002A04DA8918B9
:10A1500004390B68D01804387047000070B505004A
:10A16000080011000022064C22601A0000F03AF8A4
:10A17000431C03D12368002B00D02B6070BDC04668
:10A180008C26002058220120014B40421A60704763
:10A190008C26002058220120014B40421A60704753
:10A1A0008C26002058220120014B40421A60704743
:10A1B0008C2600205822024B00201A607047C046AF
:10A1C0008C26002058220120014B40421A60704723
:10A1D0008C26002058220120014B40421A60704713
:10A1E0008C26002058220120014B40421A60704703
:10A1F0008C260020044A1368002B03D01818106026
:10A2000018007047014BF9E77812002090260020D3
:10A2100058220120014B40421A6070478C260020D2
:10A22000FEE7C046F8B5C046F8BC08BC9E4670477D
:10A23000F8B5C046F8BC08BC9E46704766616C73B2
:10A24000650074727565006C697374206F662025F3
:10A2500064206974656D73006F626A656374206F52
:10A260006620636C6173733A2025640053746163E4
:10A270006B20756E646572666C6F77003606000041
:10A28000C8050000460600007C060000B806000075
:10A29000F20600002E070000560700009407000099
:10A2A000DA070000360800007C080000FA08000009
:10A2B000360900005E09000098090000E20900006C
:10A2C0000A0A0000420A00007C0A0000B80A0000E6
:10A2D0003E0B0000060C0000900C0000EE0C00008D
:10A2E000380D00005A0D00007E0D0000620E0000C7
:10A2F000AE0E0000360600003606000036060000EE
:10A300002A0F0000B20F00001C10000066100000B1
:10A31000B41000003A110000C21100001012000039
:10A320005A12000090120000E412000030130000E6
:10A330007C130000D81300003414000072140000D5
:10A34000DE1400001615000062150000AE150000B6
:10A35000FA1500003416000080160000D416000024
:10A360003606000036060000360600003C170000E6
:10A3700074170000AC170000DA1700001218000074
:10A3800040180000360600003606000036060000C1
:10A390003606000078180000C018000036060000DD
:10A3A000360600000C1900003A190000841900005C
:10A3B000360600003606000036060000B21900001E
:10A3C000E2190000121A0000421A0000881A000068
:10A3D000C01A0000EC1A0000161B0000401B000011
:10A3E000701B0000A01B0000CC1B0000F81B00002D
:10A3F000281C0000541C0000360600003606000031
:10A40000360600003606000036060000841C0000F8
:10A41000B21C0000E01C00000E1D00003C1D0000EE
:10A42000741D0000AC1D0000E41D00001C1E000097
:10A43000541E0000821E0000BA1E000036060000F6
:10A44000360600003606000036060000360600001C
:10A45000360600003606000036060000360600000C
:10A4600036060000360600003606000036060000FC
:10A4700036060000E81E0000161F0000070000005E
:10A48000030000006D6963726F3A6269740068616D
:10A4900073546F6E6500706C6179546F6E650068FF
:10A4A0006173536572766F00736574536572766F6E
:10A4B0000000000000000000010000000200000099
:10A4C00003000000040000000A0000000D0A564DC1
:10A4D0002050616E69633A2025730D0A00496E733E
:10A4E000756666696369656E74206D656D6F7279F6
:10A4F00020666F72204D6963726F426C6F636B737D
:10A50000206F626A656374206865617000496E73CC
:10A51000756666696369656E74206D656D6F7279C5
:10A5200020666F72204D6963726F426C6F636B734C
:10A5300020737461636B00626164206F626A65639B
:10A540007420617420256C640A0025783A20256403
:10A5500020776F7264732C20636C6173734944209D
:10A5600025640A004865616465723A2025780A000E
:10A5700009307825782C0A006D6973630068657866
:10A58000546F496E740073696E006E657400686183
:10A59000735769466900737461727457694669003C
:10A5A00073746F705769466900776966695374619F
:10A5B000747573006D7949504164647265737300FA
:10A5C0007468696E674465736372697074696F6EED
:10A5D00000636C6561725468696E67446573637289
:10A5E000697074696F6E00617070656E64546F5449
:10A5F00068696E674465736372697074696F6E0031
:10A60000617070656E64546F5468696E6750726FE4
:10A610007065727479001A1B1C03040607090A1777
:10A6200018191A1B1C03040607090A17181964696C
:10A6300073706C6179006C696768744C6576656CE1
:10A64000006D62446973706C6179006D6244697376
:10A65000706C61794F6666006D62506C6F74006D4E
:10A6600062556E706C6F74006D62447261775368EE
:10A67000617065006D625368617065466F724C650C
:10A6800074746572006E656F506978656C53656EA1
:10A6900064006E656F506978656C53657450696EBF
:10A6A00000000000000000000100000002000000A7
:10A6B0000300000004000000050000000600000088
:10A6C0000700000008000000090000000A00000068
:10A6D0000B0000000C0000000D0000000E00000048
:10A6E0000F00000010000000120000001400000025
:10A6F00016000000180000001A0000001C000000F6
:10A700001E000000200000002300000026000000C2
:10A71000290000002C0000002F0000003200000083
:10A72000360000003A0000003E0000004200000039
:10A73000460000004B0000005000000055000000E3
:10A740005A00000061000000680000006F00000077
:10A75000760000007D000000840000008B000000F7
:10A760009200000099000000A0000000A700000077
:10A77000AE000000B5000000BC000000C3000000F7
:10A78000CA000000D1000000D8000000DF00000077
:10A79000E6000000ED000000F4000000FB000000F7
:10A7A000FF000000000000000008080800080A4A36
:10A7B0004000000A5FEA5FEA0ED92ED36E193244D8
:10A7C00089330C924C924D08080000000488080858
:10A7D000040804848488000A448A4000048EC480EB
:10A7E000000000048800000EC00000000008000106
:10A7F000224488100C9252524C048C84848E1C8209
:10A800004C901E1EC244924C06CA525FE21FF01EBC
:10A81000C13E02448ED12E1FE24488100ED12ED1AB
:10A820002E0ED12EC4880008000800000480048881
:10A830000244880482000EC00EC008048244880EC0
:10A84000D126C0040ED135B36C0C925ED2521C924C
:10A850005C925C0ED010100E1C9252525C1ED01CEA
:10A86000901E1ED01C90100ED013712E12525ED26C
:10A87000521C8808081C1FE242524C125498149231
:10A88000101010101E113B75B131113935B3710C18
:10A890009252524C1C925C90100C92524C861C921C
:10A8A0005C92510ED00C825C1FE48484841252525C
:10A8B000524C1131312A44113135BB7112524C9234
:10A8C00052112A4484841EC488101E0EC808080E23
:10A8D00010080482410EC242424E048A4000000029
:10A8E0000000001F0804800000000ED2524F10101C
:10A8F0001C925C000ED0100E02424ED24E0C925CA6
:10A90000900E06C81C88080ED24EC24C10101C9225
:10A91000520800080808024002424C101498149291
:10A920000808080806001B75B131001C925252003D
:10A930000C92524C001C925C90000ED24EC2000E43
:10A94000D010100006C8049808080EC8070012525C
:10A95000524F0011312A4400113135BB00124C8C8A
:10A960009200112A4498001EC4881E06C48C848656
:10A97000080808080818080C881800000C836025CF
:10A98000642025642025642025640A00436F6D70CF
:10A99000616374656420466C61736820636F6465ED
:10A9A0002073746F72650A25642062797465732060
:10A9B0007573656420282564252529206F66202568
:10A9C00064002564202564202564202825642077E0
:10A9D0006F72647329002564207265636F726473FB
:10A9E0002C20256420776F7264732C206D61784968
:10A9F000442025642C20636F6D70616374696F6EF1
:10AA0000206379636C657320256400426164207261
:10AA100065636F726420666F756E64206475726919
:10AA20006E6720696E697469616C697A6174696FB7
:10AA30006E210A004E6F7420656E6F756768207214
:10AA40006F6F6D206576656E206166746572206338
:10AA50006F6D70616374696F6E0A00526573746F15
:10AA60007265642025642073637269707473005387
:10AA700074617274656400536372697074732063E7
:10AA80006C6561726564002D2D2D2D2D0A005065B9
:10AA90007273697374656E74204D656D6F72792081
:10AAA000546573740A0A000A496E697469616C69B5
:10AAB0007A696E67204D656D6F72790A004D656D1C
:10AAC0006F727920696E74697469616C697A656402
:10AAD0003B2077726974696E67207265636F726478
:10AAE000732E2E2E0A005265636F726420617420EB
:10AAF0006F66667365742025643A2025642025649A
:10AB00002025642025642028256420776F726473D3
:10AB1000290A0046696E616C3A2063757272656E2F
:10AB200074202564207573656420256420633020BB
:10AB300025642063312025640A00E2ECF0F4F8FC7F
:10AB400000046E756D626572006E6F6E65006F74E5
:10AB5000686572007061697200737472696E670073
:10AB6000726164696F0064697361626C65526164EB
:10AB7000696F006D657373616765526563656976BA
:10AB80006564007061636B657452656365697665C1
:10AB9000007061636B657453656E64007265636514
:10ABA00069766564496E7465676572007265636590
:10ABB000697665644D657373616765547970650086
:10ABC0007265636569766564537472696E67007354
:10ABD000656E64496E74656765720073656E645076
:10ABE0006169720073656E64537472696E67007395
:10ABF00065744368616E6E656C0073657447726F4F
:10AC0000757000736574506F776572007369676E55
:10AC1000616C537472656E677468004E6F20667263
:10AC20006565207461736B20656E7472696573006D
:10AC30004D656D6F727920636C656172656400416A
:10AC40006C6C207461736B732073746F70706564C7
:10AC50000076303634002025732025730073656E2E
:10AC6000736F72730074656D70657261747572656F
:10AC70000074696C74580074696C74590074696C60
:10AC8000745A00746F756368526561640069326359
:10AC90005265616400693263577269746500746655
:10ACA0007400656E61626C65446973706C617900F3
:10ACB000736574506978656C006C696E65007265C7
:10ACC000637400726F756E646564526563740063CB
:10ACD0006972636C6500747269616E676C6500749B
:10ACE00065787400746674546F7563686564007485
:10ACF0006674546F7563685800746674546F756336
:10AD0000685900746674546F756368507265737324
:10AD10007572650057656C636F6D6520746F204DAB
:10AD20006963726F426C6F636B73210053504943C8
:10AD30006C6173733A3A535049436C617373284E94
:10AD400052465F5350495F547970652A2C207569CB
:10AD50006E74385F742C2075696E74385F742C20A3
:10AD600075696E74385F742900705F737069202193
:10AD70003D204E554C4C002F55736572732F6A6FF2
:10AD8000686E6D616C6F6E65792F4C69627261726D
:10AD9000792F41726475696E6F31352F7061636B05
:10ADA000616765732F73616E646565706D69737437
:10ADB00072792F68617264776172652F6E524635C1
:10ADC0002F302E362E302F6C696272617269657376
:10ADD0002F5350492F5350492E63707000000000CC
:10ADE00000000000000000000B4F0000D14E0000EA
:10ADF000F74E0000014F0000314F0000F54E0000FB
:10AE00000300000002000000010000000400000038
:10AE100005000000110000000C0000000B00000005
:10AE2000120000000A000000060000001A000000E6
:10AE300014000000170000001600000015000000BC
:10AE400010000000FFFFFFFFFFFFFFFF00000000FA
:10AE50001E0000001900000018000000070000009C
:10AE600008000000090000000D0000000E000000B6
:10AE70000F0000001C0000001B0000001D0000006F
:10AE8000130000000000000000000000000030433C
:10AE900000000000000030C3FB21F93FFB21094006
:10AEA0007CD91240FB2119407A6A1F407CD922408C
:10AEB000BBFD2540FB2129403A462C407A6A2F40B1
:10AEC0005C4731407CD932409C6B3440BBFD3540FF
:10AED000DB8F3740FB2139401BB43A403A463C40B7
:10AEE0005AD83D407A6A3F404C7E40405C474140E2
:10AEF0006C1042407CD942408CA243409C6B444041
:10AF0000AC344540BBFD4540CBC64640DB8F474097
:10AF1000EB584840FB21494083F9A200444E6E00A3
:10AF2000FC291500D1572700DD34F50062DBC00095
:10AF30003C999500419043006351FE00BBDEAB009D
:10AF4000B761C5003A6E2400D24D42004906E000C8
:10AF500009EA2E001C92D100EB1DFE0029B11C0055
:10AF6000E83EA700F535820044BB2E009CE9840032
:10AF7000B4267000417E5F00D691390053833900BA
:10AF80009CF439008B5F840028F9BD00F81F3B005A
:10AF9000DEFF97000F980500112FEF000A5A8B0073
:10AFA0006D1F6D00CF7E360009CB2700464FB700DE
:10AFB0009E663F002DEA5F00BA277500E5EBC700EB
:10AFC0003D7BF100F739070092528A00FB6BEA00E3
:10AFD0001FB15F00085D8D00300356007BFC46000A
:10AFE000F0AB6B0020BCCF0036F49A00E3A91D0043
:10AFF0005E619100081BE60085996500A0145F0062
:10B000008D40680080D8FF0027734D000606310090
:10B01000CA561500C9A873007BE260006B8CC000A3
:10B020000200000003000000040000000600000011
:10B0300000000040FB21F93F000000002D44743E59
:10B04000000000809846F83C0000006051CC783B3E
:10B0500000000080831BF0390000004020257A3872
:10B06000000000802282E336000000001DF36935F5
:10B0700000000000000000000D680000FD650000F9
:10B080007D68000091680000876800000968000082
:10B09000FD6700009D68000029680000F967000056
:10B0A00058740000B6730000B6730000B47300005B
:10B0B0004A7400004A74000040740000B473000039
:10B0C0004A740000407400004A740000B473000029
:10B0D000507400005074000050740000DA740000D6
:10B0E00058800000187F0000187F0000167F0000C5
:10B0F000308000003080000022800000167F0000B9
:10B10000308000002280000030800000167F0000A8
:10B11000388000003880000038800000388200004D
:10B120002C2066756E6374696F6E3A2000617373CC
:10B13000657274696F6E2022257322206661696CC6
:10B1400065643A2066696C6520222573222C206C88
:10B15000696E65202564257325730A00430000008D
:10B160002C020020232D302B2000686C4C006566DB
:10B170006745464700303132333435363738394148
:10B18000424344454600303132333435363738395E
:10B19000616263646566000020202020202020205A
:10B1A0002028282828282020202020202020202077
:10B1B0002020202020202020881010101010101097
:10B1C00010101010101010100404040404040404DF
:10B1D0000404101010101010104141414141410170
:10B1E000010101010101010101010101010101014F
:10B1F000010101101010101010424242424242025E
:10B20000020202020202020202020202020202021E
:10B2100002020210101010200000000000000000C8
:10B22000000000000000000000000000000000001E
:10B23000000000000000000000000000000000000E
:10B2400000000000000000000000000000000000FE
:10B2500000000000000000000000000000000000EE
:10B2600000000000000000000000000000000000DE
:10B2700000000000000000000000000000000000CE
:10B2800000000000000000000000000000000000BE
:10B2900000000000000000000000000000000000AE
:10B2A000000000000000000000000000000000009E
:10B2B000000000000000000000000000000000008E
:10B2C000000000000000000000000000000000007E
:10B2D000000000000000000000000000000000006E
:10B2E000000000000000000000000000000000005E
:0CB2F00000000000000000000000000052
:08B2FC00784EFF7F0100000005
:10B30400FFFFFFFF400600008EA40000F51F0000B1
:10B3140096A40000F11F00009FA40000F91F000084
:10B32400A8A40000FD1F00007DA50000412400002A
:10B3340086A50000952400008EA50000712500005C
:10B3440096A5000089250000A0A500009325000013
:10B35400A9A500009D250000B4A50000A7250000B4
:10B36400C0A50000B1250000D1A50000BB25000048
:10B37400E7A500007F25000000A600007525000059
:10B3840036A60000E125000041A60000A12A000025
:10B394004BA60000B527000058A60000D5270000E2
:10B3A4005FA600002528000068A60000752800009C
:10B3B40074A60000CD2A000085A60000DD29000047
:10B3C40092A60000AD2900001800000066AB000042
:10B3D4001D35000073AB00003D38000083AB000056
:10B3E400DD37000091AB0000CD3900009CAB0000BC
:10B3F40039350000ACAB0000A1350000C0AB000043
:10B4040049350000CFAB0000ED3A0000DBAB000093
:10B41400753A0000E4AB0000193A0000EFAB0000FD
:10B4240055370000FAAB0000D936000003AC000029
:10B434000D3700000CAC00005135000019FCFFFF73
:10B44400FFFFFFFFFF00000065AC0000C5480000DF
:10B4540071AC0000314C000077AC0000414C00009E
:10B464007DAC0000514C000083AC0000F9480000A2
:10B474008DAC0000614C000095AC0000394A00001E
:10B48400A2AC0000ED4C0000B0AC0000F14C000098
:10B49400B9AC0000F54C0000BEAC0000F94C000053
:10B4A400C3AC0000FD4C0000CFAC0000014D000017
:10B4B400D6AC0000054D0000DFAC0000094D0000D3
:10B4C400E4AC00000D4D0000EFAC0000114D000095
:10B4D400F9AC0000E94C000003AD0000E54C0000AD
:10B4E4000300000002000000080000000A00000041
:10B4F400FFFFFFFF00000000010000000000020049
:10B5040001000000FFFFFFFF000000000200000038
:10B514000000040002000000FFFFFFFF0000000025
:10B524000300000000000800030000000000000009
:10B5340098B20000B8B20000D8B2000000000000C9
:10B544000000000000000000000000005CB10000EA
:10B5540000000000000000000000000000000000E7
:10B5640000000000000000000000000000000000D7
:10B5740000000000000000000000000000000000C7
:10B584000000000000000000000000002C02002069
:10B5940097B1000039010000A14E0000C151000024
:0CB5A400016B00000D0100000000000021
:04000003000066CDC6
:00000001FF
